:020000041100E9
:10300000002373B52B4D2C4C28006361022601F080
:1030100075F94021FE2221742800284B009601F00A
:10302000BFF9002836D1217CFF222800244B0096CE
:1030300001F0B6F900282DD1224BA2899A4226D15F
:10304000E389214A93420DD1204B6361204B2268D2
:10305000002A03D1002B01D043CB43C4280001F048
:103060008BF973BD1B4A934201D00023EFE71A4B43
:103070001A4A1B68934206D9C02304222800217CE7
:103080009B0001F003FA114B6361154BDFE700234E
:103090002374EAE7CC233821AC2228009B01217459
:1030A00001F0F4F90028F2D10E4B63610E4BE3817D
:1030B0000E4BCCE7D441FF1F9461FF1FA061FF1F9F
:1030C000A261FF1F5959000083050000294100112A
:1030D00060B9001182150000B861FF1F871300005E
:1030E0006CB90011E1410011AAAAFFFF54B9001107
:1030F000F7B5164B0192C318021D002000938823D8
:103100005B05D3181B685C1C1AD09CB2402C18D8E5
:103110008D781E0CAC466746CD782D023D43AE42FD
:1031200006D1019800280ED110000C70240A4C70B2
:1031300003249BB20733A343D218009B9A42DED3E9
:10314000FEBD4432F9E71000FAE7C046FC0F00006C
:10315000802213B503000324019189B25201073183
:103160009B18A14304305A1A88235B05C3181B68B7
:10317000591C03D190429241104016BD99B240298A
:1031800007D80B000733A343C0189042ECD30020AC
:10319000F3E74430F9E7134B134A1B68126810B584
:1031A000FA24934201D81A00F824104BE4021B6859
:1031B0009A4210D813000E4A12689A420ED3013375
:1031C00007D1F823DB029C4203D10A49054808F0E5
:1031D0009BFA200010BDFC24E402ECE7FE24E4028C
:1031E000F7E7C04600C0071100D0071100E0071143
:1031F00000F00711FFFFFF7FF0B59BB015000490B2
:103200000391402A00D9A0E006AB59801A80FFF74D
:10321000C2FF0400042816D9002206A9FFF768FFA0
:10322000052810D906AB1B88AB420CD1002D07D066
:10323000514B2A000499C01808F0FEF9002802D169
:1032400001201BB0F0BD06AB1D8020000699FFF7E2
:103250007FFF041E7BD1069B0793FFF79CFF802313
:103260005B01C618802307001B039E4201D3F8268A
:10327000F60288235B05F31801931B68013302D023
:10328000019808F0F1FA3D49019808F03DFA3B1D1C
:103290000293331D05938822029B52059B181B68DD
:1032A00008935A1C3CD044219AB20091402A04D879
:1032B0000320D11D814389B2009103991B0C8B42DD
:1032C00024D0402A22D80122300008A9FFF710FF9D
:1032D000021E1BD1380008A9FFF70AFF04000428CA
:1032E00031D9009A059B9B1880225201B218934253
:1032F00040D288235B05C118009A09A808F02CF871
:103300001D4B009A09A9F01808F076F9009A029B63
:103310009446634402931A4B029AFB189A42BAD31A
:1033200088235B05FC1821680198013908F0ECF945
:10333000200008F099FA039A07AB5A8030000799E9
:10334000FFF706FF0400002C03D1002079E70428D2
:10335000FBD988235B05E018069908F0D5F903230B
:10336000EA1C9A4300D16BE7034B0499E01808F07C
:1033700043F965E70424ECE704000011FFFFFF7F39
:10338000F80F0000F7B505001400402A21D80027E7
:1033900001AE71803780FFF7FEFE042816D93A008F
:1033A0003100FFF7A5FE042810D93688BC420BD0A7
:1033B000BD4209D0221CB44200D9321C064B92B245
:1033C000C118280007F0C8FF30B2FEBDC04300B2EC
:1033D000FBE703204042F8E70400001137B5042260
:1033E00004000D0001A81649FFF7CCFF02000428D5
:1033F0000BD1019BA34208D3AB4204D0104901A8D2
:103400000195FFF7F9FE01203EBD0E4C2368200018
:10341000019308F029FA019920000139019108F07F
:1034200073F980235B01E418074B9C42EED1042220
:10343000034901A80195FFF7DFFE0020E4E7C0463D
:103440005555000000C007110000081130B589B0C3
:1034500008F00AF810226946254808F05DF8254B67
:10346000009A9A420ED1019B029A0F2B33D8002169
:1034700001240698013B08D2002900D00292029B49
:10348000013331D10023029325E0551CF2D1020013
:103490002100EFE710341022200004A908F03CF8C6
:1034A000029B013301D1069B0293882304995B059B
:1034B000C918059B06981A03120B049105928142C4
:1034C00003D02B4201D107F047FF019B013B019341
:1034D000019B002BDED1029B002B03D004930498A8
:1034E0004168084709B030BDE025014C2D03EFE7E6
:1034F00000000111504859368022F8B5964C974B80
:10350000D200002120001C6008F046F82300944AF5
:1035100088331A60934B1A786A23002A00D011333B
:10352000E3620A232365904B37221B780820A363AC
:103530008E4B2118E361102323628D4B3B25636181
:10354000C823DB00A36123008C331A602823013ACF
:10355000E26320646364CA67043A211DCA672100DC
:10356000BC310D602100C03108602100C4310B6006
:1035700021000635CC310D602100083DC8310D60B9
:103580002100D0310A602200D43210602200D832EB
:10359000136022000227E032210017604222DC3152
:1035A0000A6021001B3DE4310D602100E831086014
:1035B0002100EC310B6023000521F4331960230056
:1035C000F0331A602300183290331A6023009433CA
:1035D000186023001E3A98331A60AF23DB00236083
:1035E000644BFA262363644B644DE360644BF03113
:1035F000A3642300FF31FC33B600A16021611E608B
:10360000A5627325E5656D3D6565A56596255D4AF1
:10361000AD00E264666258606766A566002709250A
:10362000A767E566584F594D606720002567E26738
:103630003A6015279C30676007001A203860200028
:10364000A0300700212038602000A83007004C4837
:1036500038602000F830066026006427A436376002
:1036600026005F3FAC3637602600033FB036376038
:103670002600C637B436376026000027B8363760D4
:1036800038269E60424E96205E64424E5A66DE6147
:10369000414E9A645E62F53EFF3E9E621E269A6728
:1036A000354A8000DE661F675F67DD651D6618624C
:1036B000DA67BE23394A5B00E250394BD8382350D1
:1036C00004302250C4225200A350C623E4205B00E1
:1036D000E1500433334AE1503349344BD16034492B
:1036E000800019503349E938FF3819503249043005
:1036F000195032493248D16132491163324951631C
:103700001900F4310860CE20304940001160304982
:10371000195019002F48F83108602F49D1658221CE
:103720002E4A89005A501A002D490832D1671A00D2
:103730002C49B432116088212B4A89005A501A0052
:103740002A49883211602A4ADA6407F085FF01208D
:1037500007F0EAFEF8BDC0460004FF1F3064FF1FFB
:10376000006FFF1F0444FF1F4A0AFF1F3A070000B3
:1037700080C3C9019A020000DC0500006A1800003D
:1037800050C3000088130000F009FF1F204E000006
:103790006509FF1F68100000C409000040420F00C7
:1037A00010270000FC00FF1F751CFF1F0000FF1FFB
:1037B000C92CFF1F5130FF1FE92EFF1F3520FF1FAF
:1037C0002527FF1F5120FF1FFD21FF1FC11FFF1FC6
:1037D0004929FF1F312AFF1F8D19FF1F5528FF1F81
:1037E0007925FF1F8525FF1FC11EFF1F791FFF1FA2
:1037F000391EFF1F0223F0B50124644D644E2B7067
:10380000644B91B01C70644F03933368002108200F
:10381000BB7006F00DFC082006F004FB0023984264
:1038200005D0BA78552A02D0332A00D0A1E03360FF
:10383000042006F077FD07F07FFFFFF75DFE07F03D
:10384000BBFE1F2201240021544B10AE1A70544BB2
:103850001C70544B1970544B19689143163A0A4323
:103860001A60602219689143403A0A431A6007F0CF
:103870002BFF07F039FD4D4B9847C120FF214C4BE2
:1038800080001A588A431A50C522920098588843DB
:10389000BF39014399509858464908408021C901D1
:1038A0000143802099509958C0050902090A014333
:1038B000995080214048490107F00EFF0323220060
:1038C0003E49019400933E4807F036FE2C223D49C4
:1038D00005A807F041FD05AC61782078023406F0B8
:1038E000C1FAA642F8D1384C0121002006F0CEFBE7
:1038F0000920012106F0CAFB2268344B03201A403C
:10390000A023DB0213432360802322689B0413431C
:10391000236022682E4B1A4080239B0313432360AD
:103920002C4A2D4B934200D8012007F08DFF07F061
:1039300033FD80232268DB0413432360287807F0DB
:103940003BFF039B1878C0B207F066FF07F03CFD11
:103950002249042007F0B0FD06F0B0FC00F040F86A
:1039600000F0C0FD00F068FE00F00CFA002011B07D
:10397000F0BD00932100194A042007F0FDFD8023CB
:10398000DB059C62FFF762FD52E7C0464A0AFF1F53
:1039900034F000400444FF1FC461FF1F480AFF1FAA
:1039A000490AFF1F680AFF1FBCF00040E1A20000A7
:1039B00000E100E0FF00FFFF0844FF1F8C56FF1FDF
:1039C0000854FF1F78B8001114F00040FF7FF8FF83
:1039D000FFFF9FFF0080FF1F006FFF1F3B000108DC
:1039E000002210B51100112007F036FC10BD0000B8
:1039F000F8B500230926374F374C3B62E3681120A6
:103A0000B343E36007F0A0FD112007F015FD11207E
:103A100007F0B2FC402322688025134323608023F3
:103A20006268DB0213436360A3682C4A2B43A360E4
:103A3000A36802211340A3608023A2689B01134363
:103A40001022A360236C072093432364236C0F3A56
:103A50001343236480235B003B62226B204B1A409C
:103A60002263626B1A406263A26B1A40A263E26B2C
:103A70001340E363E3681B4A1340E36006F0F2F986
:103A80000121072006F002FB174B11205A6C154349
:103A90005D6407F0F1FBFD21144B154A89005A5073
:103AA0008023C720626B5B0313436363E36880007A
:103AB0003343E3600F4B104A195811408022120221
:103AC0000A431A50802292051A6008220B4B5A634F
:103AD000F8BDC04600F000403CF00040FFFFDFFFB3
:103AE000EFFFEFFFFFFF7FFF003800400000FF1FE8
:103AF0005118FF1F00E100E0FF00FFFF000005403C
:103B000070B5284C238C002B23D0228A002A21D187
:103B1000DA0023826382A382E38223836383A38305
:103B2000E38322606260A260E2601F4D1F4A64204E
:103B3000EB8093420AD8FA220020D200934205D9A2
:103B40001B4A0A21981807F087FEC0B2002328728A
:103B5000238470BD0720E11CCA7F01320240CA776E
:103B600005D10325201DC17F01312940C1770832CD
:103B70005200A352002321001A00088A01321B18A8
:103B80000231082AF9D1221DD27F9200A350626827
:103B900023689B18A2689B18E2689B185B099BB27C
:103BA000C3E7C0460461FF1FAC61FF1FB70B0000F5
:103BB00030F8FFFF30B503A804880B20002C0ED18D
:103BC0004968074D08784978090201430A20A9424B
:103BD00005D1012120001980024B1B7A137030BDE2
:103BE000192A0000AC61FF1FF7B5150008AA168856
:103BF0004A680F4F14785278120222430A24BA42BC
:103C000014D10122DBB2019200962A0007F0A6FA35
:103C1000041E0BD1074B1B68002B07D068782A784D
:103C20000002104342425041013098472000FEBD3F
:103C3000022900003061FF1F30B50125037904001F
:103C4000BFB02B4211D00A49408806F0F3FD28424C
:103C50000BD0084B01A95B8D4D800B80064B0022D9
:103C60001B7A60880B7103F0C5FE3FB030BDC046C3
:103C70002861FF1F4840FF1FAC61FF1F10B50549B9
:103C8000054806F08DFD0421044A054806F04AFD6A
:103C900010BDC0462861FF1FFFFF0000A4B800113F
:103CA0004840FF1F10B5024804F026FD10BDC04675
:103CB000393C0011012303700B4B1A7A4270022227
:103CC00082709A78C270DA780271032242711A798E
:103CD00082715A79C2710C2202729A794272DB792E
:103CE00083720B207047C046AC61FF1F022310B5E2
:103CF0000370013B43700533837010330371443B01
:103D000043712A3383714433C37100230372064B1A
:103D100004001B8843720A30FFF7CCFF831D0A3072
:103D2000C0B2E37010BDC046AC61FF1F10B51420D7
:103D300007F0D2FB124B14220021186007F02CFC74
:103D4000002007F049FD012007F0DEFB022007F00C
:103D50001BFD032003F074FF042005F089FF0520FC
:103D600003F0B2F9062003F07FFE072001F016FAF7
:103D7000082006F0B7FC092000F0E8FF10BDC0469F
:103D80003461FF1F07F088FA012007F0B5FC07F047
:103D900023FB0000094B10B50400984205D001290F
:103DA00004D12000064906F0FBFC10BD0229FCD11D
:103DB000013904F05FFC0028F3D0F6E7FEFF0000B5
:103DC0005A61FF1F70B50D7A100004AA2C001688E6
:103DD00010221440154220D1002E20D10A78022A48
:103DE00018D14A68517815780E4A09022943914240
:103DF00005D00D4A914209D01C800A2404E0142207
:103E00000A491A8007F0A8FA200070BD0C22084960
:103E10001A80F7E71C800124F6E70824F4E70B2456
:103E2000F2E7C046F3FF0000F4FF00009042FF1FDE
:103E300084B9001110B504000749084806F0B0FC29
:103E4000074804F099FB0020E40704D50721054A40
:103E5000054806F067FC10BD5A61FF1FFFFF000018
:103E6000953D0011E8B800118C40FF1F00B50C4BC8
:103E7000BFB01A780B4902A800F098FC6B4680B2DC
:103E8000D880002809D06A46074B01A91B88938077
:103E9000064B0022188803F0ADFD3FB000BDC046C0
:103EA0003861FF1F3961FF1FE640FF1FF041FF1F10
:103EB00000B50C4BBFB01A780B4902A801F0E0FC2A
:103EC0006B4680B2D880002809D06A46074B01A90A
:103ED0005B8D9380064B0022188803F08BFD3FB06A
:103EE00000BDC0466261FF1F6361FF1F8C40FF1F62
:103EF000F041FF1FF7B50E00377A1C0008AB110028
:103F00003D001A8820231D401F423CD13378022BEC
:103F10003BD173681F785B781B023B431E4FBB424B
:103F200008D01E4FBB4214D01D4DAB4221D00A25F4
:103F30002800FEBD002A2AD1142C2AD82200F068BD
:103F400007F00AFA174B1C70012CF1D9FFF7B0FFEC
:103F5000EEE7002A1BD1202C1BD82200F06807F0C6
:103F6000FBF9114B04211C70104B187807F074FA00
:103F7000DEE7E3B20124009201940A00310007F069
:103F8000EDF80500D4E70825D2E70125D0E70B2599
:103F9000CEE70D25CCE7C046F3FF0000F4FF00009C
:103FA000022900006261FF1F3861FF1FE461FF1FEB
:103FB000332310B5040003700A220749013007F0CB
:103FC000CBF9064B0F201B681A0AE37222731A0CF6
:103FD0001B0E6273A37310BDAC61FF1FD461FF1F82
:103FE00030B5012503790400BFB02B4213D00B4933
:103FF000408806F01FFC28420DD06A46084B02A8F4
:104000001B889380FFF7D4FF6B46D880002260881E
:1040100001A903F0EFFC3FB030BDC0465A61FF1F5D
:10402000E640FF1F10B5024804F066FB10BDC04615
:10403000E13F001170B5160004AA148805AA15788E
:104040004A685078117800022A4A084380180528E7
:104050004BD807F029FA03131E29343F0720042CFC
:104060000BD80522121BAA4200D92A0022491A8025
:104070003000091907F070F9002070BD0720112CDD
:10408000FBD81222121BAA4200D92A001B491A800F
:10409000EEE707200E2CF0D80F22121BAA4200D9FF
:1040A0002A0017491A80E3E70720032CE5D80422E9
:1040B000121BAA4200D92A0012491A80D8E7072009
:1040C000032CDAD80422121BAA4200D92A000E4976
:1040D0001A80CDE70720032CCFD80422121BAA4256
:1040E00000D92A0009491A80C2E700220A201A8052
:1040F000C3E7C046DCD5FFFF33B900118061FF1F65
:1041000023B900111EB9001119B9001114B9001119
:1041100010B50D21024A034806F004FB10BDC0464D
:1041200008B90011FC40FF1FF0B50024274E85B0F0
:104130003000B47100F0E2F8254D264BEA89297C65
:104140009A422FD10423300003AA00F057F904004B
:10415000300000F011F90123B371002C34D16B460B
:1041600099892B68C9BA4B4329891B4A1B145B18D0
:1041700053806B46D9896B6849BA89B24B436989C8
:104180001B0C5B181548191C1BB2834200DD011C77
:104190000B0400D500211388918001331380200087
:1041A00005B0F0BD0227220003AB3000009700F0FD
:1041B000F7F80E230400297C0122300000976B449D
:1041C00000F0EEF80443C3E71C00E8E7D441FF1F0A
:1041D0009461FF1F83050000AC61FF1F0F270000E3
:1041E00073B5234E300000F089F8224D07236A464C
:1041F0003000297C00F002F904003000002C33D19B
:104200006B461B787F2B2FD800F0B6F86B46D8781A
:10421000F02302041B031A406B469B8816495BBAC5
:104220009BB21A432B68000953432A891B0C9B1825
:104230004B806B465A789B7812031B011A436B68BC
:10424000024353436A891B0C9B180C481A1C1BB26F
:10425000834200DD021C130400D500220B888A80F3
:1042600001330B80200076BD00F086F80124F9E7C9
:10427000D441FF1F9461FF1FAC61FF1F0F27000097
:1042800070B5114C237C002B0FD0382B0ED10F4D65
:10429000280000F033F8CC23AC222800217C9B01BD
:1042A00000F0F4F8280000F067F870BD084BE289D0
:1042B0009A42FAD1054D280000F020F8002228008B
:1042C000217C00F0C5F8EDE79461FF1FD441FF1F8A
:1042D0008305000010B5084B1A7C002A09D05B69E1
:1042E000002B06D09847041E01D0FEF789FE20005F
:1042F00010BD0124F9E7C0469461FF1F70B5C17974
:1043000005000C00631E9C411A4BE402E4184900AE
:104310000460C9B2007905F0EFFEE97968794900D7
:104320000131C9B205F0E8FEE8790930C0B207F002
:1043300023F80023E36661332360AA795B3B002AFC
:104340000ED022689A43023B134323600A23E361A1
:104350000733236200232363A3630133E36370BD48
:1043600022689A4302231343236046236361063382
:10437000A361EFE70050004070B50025040003681A
:10438000DD66C0790930C0B207F0DEF82900207977
:1043900005F04EFE2900607905F04AFE70BD000070
:1043A000F8B51E0006AB1D78002304681700E3660D
:1043B000616007F059F801238022E3662B00276132
:1043C0005200013B08D207F027F808200A4A11687A
:1043D000002D03D12800F8BD2261F2E7236F0342CC
:1043E00003D02369013D3370013613685B1A032B38
:1043F000EED90125EEE7C0466008FF1F70B51C002E
:10440000002305681600EB66696007F02DF80123AC
:104410008022EB6623005200013B08D206F0FCFF2D
:1044200008200A4A1168002C03D1200070BD2A61BF
:10443000F2E72B6F034203D02B69013C3370013646
:1044400013685B1A032BEED90124EEE76008FF1F07
:10445000002370B504681500E366616007F004F896
:104460000123E366256106F0D7FF8020064A80001D
:104470001168636B034205D113685B1A032BF8D9EB
:10448000012070BD0020FCE76008FF1F70B51D0013
:10449000002304681600E366616006F0E5FF01236F
:1044A000E36626610F33626B1A42FCD02B0A23614C
:1044B0001023626B1A42FCD0EDB2256106F0ACFF0E
:1044C0008020074A80001168636B034205D113689E
:1044D0005B1A032BF8D9012070BD0020FCE7C04611
:1044E0006008FF1F10B5084CE368002B08D180223C
:1044F000064B52021B689B186360054B1B682360C8
:1045000006F0EAFEA06010BDD461FF1FC8F00040B5
:10451000CCF0004070B5184A936A916A9942FBD179
:1045200016498A689A421FD39A1A8B60144B012647
:10453000186893B2D202D20E4343424300204C6823
:104540001B0A1B1912029B180E4C0A684B60551C63
:10455000A3420CD8002801D04B600A600A4A1360BD
:1045600008680A4B186070BD581E821ADDE7084AB9
:1045700030009B182A00EAE700F00040D461FF1FDA
:10458000140AFF1F40420F00C8F00040CCF000406A
:10459000C0BDF0FF70B51F4C23793F2B01D93F23DD
:1045A00023711D4B22791A701878C0B206F04CFEA8
:1045B00018231A491A4A0B801A4913800B8053801A
:1045C000A379194980200B800C21938001334B4340
:1045D000164D191C0001834200D9011C2980D1808D
:1045E0006379002B11D101336371237A012B01D838
:1045F000022323726279237A0D4853430A215843D8
:1046000007F02AF90B4D286070BDA02BEDD9A0232F
:10461000EAE7C046C861FF1F480AFF1FEE41FF1FBF
:10462000B043FF1FEC41FF1FEA41FF1FE841FF1F9E
:1046300071020000B861FF1FF8B516210020FEF7D7
:10464000CDFE114C011E114D09D10C22104BC1CBD6
:10465000C1C4280006F0A0FFFFF79CFFF8BD0C22A4
:1046600020000C49FEF78EFE0C2802D0084B43CBED
:1046700043C40C2228000849FEF784FE0C28EBD026
:104680000C220021E5E7C046C861FF1F9461FF1FAF
:1046900078B90011FC0C0000F50C0000F0B51D4CC1
:1046A0008022A5440400882069465201400506F096
:1046B000BBFE902212016A441300200032C832C3AC
:1046C00016C816C38023144C144FA6689B033343AB
:1046D000A3603B6007F028F88823A0685B05C0183A
:1046E00007F0C2F80025882329008022A0685B0516
:1046F000C01840196944520006F07EFF802301353E
:10470000FF355B019D42EED1A6603E60044B9D44A7
:10471000F0BDC046FCEFFFFF2043FF1F9808FF1FBE
:1047200004100000F0B5040087B0002825D06846CA
:1047300006F062FE1B4C022806D1062269462000C4
:1047400006F07AFF002816D06946002301250F26BF
:104750002F00E25C013310091030874038002F0031
:10476000324097403A0002434A610439062BEFD1A8
:104770006846FFF793FF07B0F0BD182269460A4864
:1047800006F052FE6A46A300D358013305D0182222
:10479000FF21684606F000FFEAE70134062CF1D15C
:1047A000E9E7C0466509FF1F00090011F0B50025C3
:1047B00004000E0085B0AA4200D183E04B1C0878AB
:1047C00001934B788978377909021943F3783F06CA
:1047D0001B040B431F43039720706570252800D1ED
:1047E00093E033D8112813D806F086FE66000D0139
:1047F0000D010D010D01A700B500AE000D010D0169
:104800000D010D010D010D010D010D01E700070165
:10481000232800D1C0E0DB2800D016E1042A00D80C
:10482000A9E01025052A05D0551F2A003800711D62
:1048300006F092FD05223100200006F08DFD2A00D1
:104840003900601D06F088FD05353BE0562856D03E
:1048500010D8332800D19AE0552836D02628DAD14E
:10486000894B2900132218001D0006F095FEFEF763
:10487000C7FB59E0712800D174E0722800D17DE0B7
:10488000DC28C8D1022A00D875E07378BFB2637003
:10489000B378A370032A05D0033A390092B2F01C12
:1048A000FEF7AAFC10223900E01CFEF76BFDC51CC8
:1048B000002807DA60705CE00C222000734906F0E3
:1048C0004BFD0C25280005B0F0BD013A704D0C2AB7
:1048D00013D8002A0AD02800019906F03DFDFFF701
:1048E00059FE0C2228006B49FEF786FC29000C2299
:1048F000601C06F031FD0D25E4E70C22EBE7644D6A
:10490000654B2A0043CB43C2E9E7013A5E4D0C2ACE
:1049100011D8002A08D00199280006F01DFD0C22AC
:1049200028005E49FEF768FC29001322601C06F08F
:1049300013FD1425C6E70C22EDE705225849601C3B
:1049400006F00AFD0625BDE712225649601C06F056
:1049500003FD1325B6E708225349601C06F0FCFC52
:104960000925AFE77178F02905D8504B188801F078
:10497000E3FB0225A6E7FF236370FAE74C4B012A0D
:1049800003D072785A706270F3E75B78F4E7200026
:10499000FFF70EFB050095E7042A04D9454D2F606B
:1049A00006F09AFCA860FFF7B5FD0422039003A966
:1049B000601C06F0D1FC052584E73F4D062A15D979
:1049C00006222800019906F037FE00280ED00622A4
:1049D0000199280006F0C0FC062238492800FEF79D
:1049E0000BFC0123324A51780B43537029000622F5
:1049F000601C06F0B1FC072564E7012ABBD0707883
:104A0000FFF790FEB5E7012800D004E7931E2C4F76
:104A1000132B04D87378002B09D100F009F9294B26
:104A200039001D78601C6A1E06F096FC4AE7551E88
:104A30002A000199380006F08FFC2349AAB23800F9
:104A4000FEF7DAFB00F02CF9E9E7DA2893D1042A23
:104A500091D9082A15D9B37972791B021343F279D7
:104A600012041A43337A1B0613433B603B6805224A
:104A700031002000039306F06FFC0422601D03A99F
:104A80006CE7FE236370F1E79461FF1F84B90011A6
:104A9000C861FF1FFC0C000078B90011F50C000084
:104AA000A061FF1F8061FF1F2443FF1FF041FF1F14
:104AB000C461FF1FD461FF1F6509FF1FADAC00007B
:104AC000C563FF1FC363FF1FAEDE00007047000019
:104AD000020010B5094B0A32094C92B2DA815A82AF
:104AE00098811882207802F08DF90422054B01216B
:104AF00020781A7006F0B0FC10BDC046AE42FF1F11
:104B00000E64FF1F0D64FF1F013870B5042809D81B
:104B100006F0CAFC0309230812001E4B0221187874
:104B200006F09AFC70BD1B4B0821187806F01CFC9F
:104B30000022194B1A72F5E780220024164B154DFE
:104B400052001A81082128781A68DC7206F07CFC71
:104B50002100287806F098FCE4E70E4B082118782D
:104B600006F002FC0D48FFF7C1F80D4B0D4A9B798A
:104B700093800D4A13800022074BDA720132FF3214
:104B80001A810A4B5B78002BCCD0094A136006F0DF
:104B90004BFEC7E7E461FF1FB861FF1FF941FF1F2C
:104BA000C861FF1FB043FF1FEA41FF1FC461FF1F21
:104BB00034F0004010B5002905D1082803D1013197
:104BC000013005F063FA10BD10B501290FD1082896
:104BD0000DD10021013005F059FA054B1B78002B4F
:104BE00005D02622034B04485A72FFF771FF10BD0F
:104BF000E663FF1FB861FF1FC40900000300F0B5A2
:104C00000A4D8E18B14202D152008018F0BD0C78C6
:104C10002F6824093C5D0F271C700C7801313C4043
:104C20002F683C5D5C700233ECE7C046E441FF1F37
:104C30000E22124B10B51A700D23114C114923701E
:104C4000093A043B1048637006F086FB2D230122CD
:104C50000E490F48E371FFF7D1FF01220D49FFF71D
:104C6000CDFF01220C49FFF7C9FF030000200B49CB
:104C700002001870FEF7C0FA10BDC046E263FF1FC5
:104C8000C363FF1F33B90011C563FF1F6709FF1F0F
:104C9000CB63FF1F6609FF1F6509FF1FAEDE000023
:104CA00070B5124C142220001149FEF76BFB431E15
:104CB000104D132B17D8AB78002B14D0431C2B703E
:104CC00009236B7000230019037028782900013034
:104CD000C0B206F009FC297822000139C9B20020CF
:104CE00005F03EFC70BDFFF7A3FFEEE7C563FF1FB5
:104CF000AEDE0000C363FF1F10B5114B1A781870A9
:104D0000002A0ED000280BD10E4B1A78062A07D89D
:104D10005423D340DB0703D50B4B187802F072F80D
:104D200010BD0028FCD0074B1B78012B02D0033BA1
:104D3000022BF5D8044B0121187806F08DFBEFE724
:104D4000E663FF1F0D64FF1F0E64FF1F70B5504E1A
:104D5000504A51493070082005F08EFA012109208F
:104D600005F094F9092005F075FA0121002005F0FD
:104D70008DF9002005F06EFAFEF742F906F024FCEA
:104D8000032246494648FFF739FF2D240300042239
:104D90001C7044490130FFF731FF30230470424D4D
:104DA000424C437083702E3B062220004049EB8723
:104DB000FEF7E8FA062813D0200006F01DFB0228B3
:104DC00009D00321200006F04FFC8D23E3706E3BD9
:104DD000237119336371062220003549FEF70CFA5E
:104DE000344B1B68FC335C64FFF75AFF0020FFF76D
:104DF00083FF314C314A0121314B1278207801F088
:104E0000C3FF304A304B12780021207801F0BCFFFC
:104E100001222E4B1A702E4B9B78552B31D12D4BE6
:104E20003B325A722C4B2D4AAB81EA812B826A822B
:104E30002021307806F088FA0120404205F0DCFBA2
:104E40000120404205F078FCFFF762F9FEF716FFFB
:104E500000F0AEFC01204042FEF7ECFF012006F01E
:104E6000E3FBF02001F04CF90121307806F0F4FA70
:104E7000307802F023F91A4806F09EFAFEF7B8FDE2
:104E800070BD6422174B5B7953431A000A32CBE79B
:104E9000E461FF1FB54B0011C94B00112443FF1FF4
:104EA0008061FF1FA061FF1FAE42FF1F6509FF1F4A
:104EB000ADAC00003064FF1F0E64FF1F1842FF1FDF
:104EC000F941FF1FE263FF1FC363FF1FB463FF1FAE
:104ED000C461FF1FB861FF1FC4090000CE090000B4
:104EE000E661FF1FC861FF1FF8B50A0020230D000F
:104EF0001A4019425DD05C4B1B78002B42D0FFF763
:104F000009FB5A4B5A4C5B4E99686268737A8A1A4D
:104F1000DB039A4202D36160FEF76AFD327A217A9E
:104F2000531EDBB2994230D1FFF7AAF9637A002B06
:104F300025D0013BDBB26372002B20D14E4B9B7816
:104F4000552B01D106F070FCE37A002B12D0002320
:104F5000A27AE3729A4202D0A372FEF7D1FD474AC9
:104F6000474F1388380001331380FEF7BFFE390026
:104F700006F07AF9642370795843FFF7A9FD237A84
:104F80000133237220206840F8BD9142CED3002720
:104F90002772FFF79FF9A37ABB4202D0A772FEF7F0
:104FA000AFFD374F3800FEF7A1FE390006F05CF97F
:104FB000BCE70BB2002B0ADA324B187806F024FC5F
:104FC000002801D006F0D0FA80200002DBE702249E
:104FD000214206D0264B01201A72FFF78DFE2000D9
:104FE000D1E70B071BD5FFF795FA204B2049214C41
:104FF00098684A68637A821ADB039A4202D348604F
:10500000FEF7F6FCFFF766F9FFF73AF900F0EAFB66
:105010002368DB0701D5FFF705F80820B3E7102365
:105020000E001E40194209D0FEF76AFD0E4B1B7898
:10503000002B01D1FEF736FE1020A4E70124214207
:1050400009D0114800F06EF806F01EFB310009206F
:1050500005F01CF8C3E7042408002040214200D1D9
:1050600092E7FEF703FFBAE7E663FF1FD461FF1F75
:10507000B861FF1FC861FF1FC461FF1FAC61FF1F44
:10508000F941FF1FE461FF1FDC41FF1FF0B51B4B1F
:105090001B4F1B883A8804001A4E1B4D85B09A425C
:1050A0000DD832889A420AD3184B1A882B889A4214
:1050B00005D1174A174B12881B889A421BD005202E
:1050C00001F074F83B8802AA138033880190538062
:1050D0002B88114D93800F4B02A91B88D3800F4B57
:1050E0002A78188802F090FD0D4B08212878019A43
:1050F0001C7006F071FA05B0F0BDC046B263FF1F28
:10510000EE41FF1FEC41FF1FEA41FF1FB063FF1F8D
:10511000AE63FF1FE841FF1F0E64FF1FF041FF1F3A
:10512000AC63FF1F13B50C4B1C78002C11D1002869
:1051300001D00A4B18600A4A0A4B11780A4A1078C3
:105140000A4A01920A4A0092002205F001F9200061
:1051500016BD1124FBE7C0460D64FF1FA863FF1FA7
:105160000C64FF1FFC63FF1F0E64FF1FE863FF1F3B
:10517000EC63FF1F10B5064B12201B78052B06D1E0
:10518000044B13221988044B187801F0EBF910BD79
:105190000D64FF1FF041FF1F0E64FF1F10B50024B8
:1051A0000122114B52421870104B1C70104B1A8088
:1051B00001F084FF04220F4B21001A700E480C32BC
:1051C00006F042FA102221000C4806F03DFA0722B0
:1051D0000B4B1C600B4B1C700B4B1C700B4B1A7059
:1051E0000B4B1C7010BDC0460E64FF1F0D64FF1FEB
:1051F000F041FF1F0C64FF1FFC63FF1FEC63FF1FE8
:10520000E863FF1FC263FF1FC163FF1FF241FF1F5F
:10521000C063FF1FF8B5174C0600257806A81424B4
:105220000078052D23D1B41F134FA5B21824BD4219
:105230001DD88D1FADB2BD4219D8FA256D00AA4206
:1052400015D21D000D4F0A3DADB2BD420FD80C4C1A
:1052500026800C4C21800C4900240A800B4A1380C4
:10526000FFF714FF0A4B0421187806F07DF82000A0
:10527000F8BDC0460D64FF1F790C0000750C0000DE
:10528000EE41FF1FEC41FF1FEA41FF1FE841FF1FF6
:105290000E64FF1FF0B50BB20D0089B0002B00DBD0
:1052A00070E1A44E307806F0AFFA041E50D00378B7
:1052B000A22B00D122E1D02B1AD0912B45D14378DB
:1052C0000E2B42D19C4B82889A423ED19B4A8368E6
:1052D0001278052A39D1032018567F2835D0984BEB
:1052E0001B68002B31D05B68002B2ED098472CE038
:1052F0008078072829D806F0D7F80428183F3F748B
:10530000A8D86378002B0CD101218C4B19708D4BE0
:105310001A78002A5BD08C4B307801F035FD0028DC
:1053200055D00722854B1A7051E061780029F8D1D9
:10533000E378002B11D0854A854B1278307801F044
:1053400023FD60706378002BEBD1200006F00CF990
:1053500080200002684009B0F0BD784B1B78022B1A
:10536000F3D00121307806F02FFA0028EAD101218C
:10537000307806F071F8E5E76378002BD1D16F4FF4
:10538000032807D13B78052B02D101333B701EE087
:105390000223FBE76F4B1A886F4B0293002A0BD056
:1053A0001B78002B03D00121307806F015F93B78EB
:1053B000062B04D1013BE9E7029B1A70F7E7042BA7
:1053C00041D10121029B3078197006F045F85C4B01
:1053D0001B68002BB9D01B68002BB6D0574A107839
:1053E00084E76378554F002B27D10622211D5B48A7
:1053F00005F0B2FF62895A4B5A491A80A2895A4B6A
:105400001A80E3890B800521397058490A80584A6F
:105410001380228A574B1A80574B1B78012B09D1D6
:105420001F2000F0C3FEFA2292004243042130788C
:1054300006F0D2F80022484B75E7312B00D070E718
:105440000022454B1A700323A0E70622002143489F
:1054500006F0FAF80023454A04211380444A3078C4
:105460001380444A138005F07FFF0821307805F04F
:105470007BFFA379083B5A425341304A03331370F0
:10548000304B1B78002B06D0334B30781A78002A2B
:1054900006D001F0B7FC0122314B52421A8096E748
:1054A0000121197005F0D8FFF5E70821307805F0E3
:1054B0005BFF6378002B00D047E72C4B2D4F029306
:1054C000E388029A04211380294B307803932389BF
:1054D000039A138063893B8006F076F9002800D098
:1054E00033E7264B1B68002B00D12EE70399029867
:1054F0003A88098800881B68984726E74379132B68
:1055000000D022E70389012B0AD11D4B1B78022B07
:1055100006D10821307805F027FFFFF72BFE14E7AE
:10552000052000F043FE08210200307806F054F810
:105530000BE7C0460E64FF1F051400000D64FF1F3B
:10554000A863FF1F1842FF1FF941FF1FE263FF1FFF
:10555000C363FF1FE463FF1FE663FF1FB563FF1F05
:10556000F041FF1FBC63FF1FBE63FF1FB263FF1F3D
:10557000B063FF1FAE63FF1FB463FF1FA463FF1F71
:10558000AC63FF1F8020C001014200D0E2E6CB07E0
:1055900031D5324B1B78002B1DD0314E05AC337802
:1055A000052B1AD1023B23702E4B21001B7823724E
:1055B0002D4B1B7863722D4B187801F089FB002866
:1055C00009D007202A4B30701B68002B03D01B68C2
:1055D000002B00D098470120BCE60E20254B062268
:1055E0001B7825492370254B1B78637002ABC018CC
:1055F00005F0B2FED8E7022308001840194209D08E
:10560000174B1B78052B03D11D4B188805F0FCFFA9
:1056100002209FE60424214203D0FFF737FD20003B
:1056200098E6082308001840194200D193E6154B6C
:105630001C78012C03D0022C0DD008208AE6124BD6
:10564000124A134913481B8812880988008800945D
:10565000FFF7E0FDF1E7FFF78DFDEEE7E663FF1FE3
:105660000D64FF1FF241FF1FC063FF1F0E64FF1F89
:10567000A863FF1FC263FF1FF341FF1FC163FF1F2A
:10568000F041FF1FAC63FF1FE841FF1FEA41FF1F0E
:10569000EC41FF1FEE41FF1F10B502A804880B204C
:1056A000002C10D1496808784978090201430C4858
:1056B000814209D1022119800A4B59881170DB7887
:1056C00000205BB2537010BD074C0A20A142FAD1F2
:1056D00002211980034B998811705B79F0E7C0466D
:1056E0006E2A0000AC61FF1F6F2A0000F7B515009D
:1056F00008AA16884A680F4F14785278120222437B
:105700000A24BA4214D10122DBB2019200962A0087
:1057100005F024FD041E0BD1074B1B68002B07D09E
:1057200068782A780002104342425041013098477D
:105730002000FEBD022900002064FF1F30B50125B6
:1057400003790400BFB02B4225D01449408805F0EE
:1057500071F828420CD0124B01A95B8D00220B80FE
:1057600002234B800F4B5B888B80608802F042F9EC
:105770000D49608805F05EF8C0070CD50B4B01A9F8
:105780001B8800220B8002234B80064B9B888B805A
:10579000608802F02FF93FB030BDC0461864FF1F8B
:1057A0001C42FF1FAC61FF1F1064FF1F7642FF1FEA
:1057B00010B5074C0749200004F0F2FF200006490D
:1057C00004F0EEFF0721054A054804F0ABFF10BDC9
:1057D000FFFF00001864FF1F1064FF1FA4B9001131
:1057E0001C42FF1F10B5024802F086FF10BDC046E4
:1057F0003D5700110200F0B501270A480A4E511822
:105800008B1A002B00DCF0BD082415784308684093
:1058100038404000805B013C58406D08002CF5D1B9
:105820000132EDE7FFFF0000BEB90011F0B5002521
:105830000F269D4200DBF0BD4C5D0709444034401B
:10584000A400A05801357840F3E70000F0B589B016
:105850006A460D000B000F27110010351C7801332C
:10586000260024093E40167054700232AB42F5D136
:105870002023024AFFF7DAFF09B0F0BDC4B90011D6
:10588000F0B54E780B7889B036020C001700019005
:105890001E43012A61D9954B9E4200D877E001331F
:1058A0009E421CD1062A17D1CA788B7812021A435D
:1058B0000B791B0413434A7912061A438C4B5A6125
:1058C00000221A705A808B4A5A608B4A9A608B4A1F
:1058D000DA60002009B0F0BD88225205EEE7884B5F
:1058E0009E423CD182498B78002B00D0F6E00C2AF6
:1058F00031D10F22A3789343E27812021343227925
:10590000120413436279120613434B60E279A079C3
:1059100012020243207A00041043627A1206024304
:10592000CA60E27AA07A1202024376484A81834230
:1059300008D804236E49142201980B7005F00CFD61
:105940001420C7E71201D21889235B059A42F0D8C8
:1059500001238B70BDE7022AFAD00523EAE76A4AE1
:1059600001239642E6D1FFF705FC052F0CD9E37819
:10597000A2781B021343227912041A4363791B068F
:105980001343624A0393136005F04EFFA1E7584D9D
:105990002B78002B9DD1AB78002B00D1A0E02B8978
:1059A00001339BB20093B34200D091E0132AD4D9C3
:1059B000CF7C8B7C3F02122120001F43FFF71AFF90
:1059C000874200D08EE0002E3DD1E378A2781B0202
:1059D00013432279E96812041A4363791B061343BF
:1059E00003930A228B4212D1FF23A370E370237129
:1059F00063716B89002B09D1E37B227C1B021204AB
:105A00001343A27B13431B0901336B8100226B8973
:105A1000002B8ED0002A67D1686837013818000B38
:105A20006B6900030390984205D9686105F01CFF7B
:105A3000EB780133EB7068681022A11C381805F070
:105A4000DBFD2E8145E76F89009A7B1E9BB2934256
:105A50003AD1E278A37812021A43237905A81B04ED
:105A6000134362796C6812061A43EB680092039242
:105A7000211D0C22049305F06FFC0120260004A9CF
:105A800040421036FFF7E2FE013F012F17D1009A86
:105A90000B232861824200D04CE704221C492000DD
:105AA00005F0AAFD042203A9686805F0BDFCE968B9
:105AB000039AFF23914200D13CE7F73B3AE73100DC
:105AC000FFF7C4FE1036DFE70923B742A4D831E759
:105AD000009BB34200D9FCE607232BE7022329E70A
:105AE000032327E7062325E70A2323E7FFFE000019
:105AF0009042FF1F00000111FFFF0000504859367F
:105B000001FF0000FFFF001102FF000034F0004021
:105B10009C42FF1F10B5034C0B000122210000F036
:105B20006BFA10BDD55C00110B8870B506000D0036
:105B30000224162B11D92B000322094900F05CFA2C
:105B4000041E0AD1074B2A881B88191C934200D9CE
:105B5000111C300089B200F0EFFA200070BDC04681
:105B6000015D00113664FF1F10B54A780400013A48
:105B70000B000220012A07D80A78002A04D0052247
:105B80002000024900F038FA10BDC0462F5D001118
:105B90000A7810B50B0004000220002A04D0072266
:105BA0002000024900F028FA10BDC046DB5D00115C
:105BB0000A7810B50B0004000220002A04D0092244
:105BC0002000024900F018FA10BDC046415E0011E5
:105BD00010B5034C0B000B22210000F00DFA10BD94
:105BE000715E001110B5034C0B000D22210000F076
:105BF00003FA10BDE35E001110B5034C0B000F2239
:105C0000210000F0F9F910BD3D5F00110A7810B5D0
:105C10000B0004000220002A04D0112220000249B7
:105C200000F0EAF910BDC0464D5F0011002310B529
:105C30001322190000F0E0F910BD000010B5034C6C
:105C40000B001722210000F0D7F910BD9F5F001153
:105C5000002310B51922190000F0CEF910BD000084
:105C600010B5034C0B001B22210000F0C5F910BD3C
:105C7000D95F0011F7B584890D0006000121002CC1
:105C800022D000238268D3561778002B1EDA0C2C02
:105C90001AD90C3CA4B2131940880093230002F0D7
:105CA00086FE431E984101307B06DB0F6B703F235D
:105CB000013C1F40A4B22870AF70AC80002C07D00C
:105CC000B3680133AB6000210800FEBD0020EBE7A4
:105CD000AC60F8E70B7803704B8843704B881B0A65
:105CE00083700B79C370042070470420022B06D107
:105CF0000020537811781B02009A0B4313807047E1
:105D00000B8803700B881B0A437002207047042025
:105D1000009983420AD1537810781B0203430B8009
:105D2000D37890781B02034300204B807047F8B56E
:105D30000D004B7801240021461C03702B788B4208
:105D400001D82000F8BD6B78B01C4F1C012B10D17E
:105D5000890069184B88022233704B88B9001B0AEE
:105D60007370691805F0C0FC04360434A4B2F9B2AB
:105D7000E4E7122359436B185A88043132705B8868
:105D800010221B0A7370691805F0AEFC123612342B
:105D9000ECE770B5049D14001E00052B01D804200B
:105DA00070BD637812781B0213432B80E378A278CE
:105DB0001B02134302226B802A71211D681D063EBF
:105DC00005F092FCB2B22A81E92AE8D82800A11D88
:105DD0000A3005F089FC0020E2E7002310B50A78BC
:105DE0009A4201D8900010BD9A008A185488013355
:105DF00004705488DBB2240A4470948884709288BA
:105E0000120AC2700430EAE710B51100029C062B9A
:105E100004D004201022142B01D010BD02222271C4
:105E20004B7808781B0203432380CB7888781B02C9
:105E3000034363800431601D05F056FC0020ECE74D
:105E400010B50C788B7804315C43E4B20370220007
:105E5000013005F049FC601C10BD0420022B06D166
:105E60000020537811781B02009A0B43138070476F
:105E700010B50C000A88023105F036FC208810BDF0
:105E800070B504000D0004981100012B01D8042006
:105E900070BD167852781202324302800200F1324D
:105EA00055701470E125002C00D10C35023B9AB2DC
:105EB0004280AA42EBD80231043005F015FC0020E4
:105EC000E6E70420009983420AD1537810781B0238
:105ED00003430B80D37890781B02034300204B8050
:105EE000704710B50C000A88023105F0FDFB2088D0
:105EF00010BD000070B501211E000420049C0E405E
:105F00000B4218D1CB40DDB28D4214D90A49DBB225
:105F1000098899420FD32300EE331D7033005800D7
:105F200011184978165C0902314301332152D9B264
:105F30008D42F4D8002070BDA842FF1F10B50C00A0
:105F40000A88023105F0D0FB208810BD10B50C780E
:105F50008B7804315C43E4B203702200013005F019
:105F6000C3FB601C10BD10B511000298032B01D8B3
:105F7000042010BD14785278043B120222430280A0
:105F8000CA788C781202224342809AB28280EB2A2D
:105F9000EED80431063005F0A7FB0020E9E710B584
:105FA0000C000B8803700B881B0A43704B888370AE
:105FB0004B881B0AC3708A880430063105F094FBB5
:105FC000A088043080B210BD0420012B03D1002032
:105FD0001378009A1370704710B50C000B8803708B
:105FE0000B881B0A43704A880230043105F07CFBA1
:105FF0006088023080B210BDF0B589B003931E4BAB
:10600000029242000700D05A019102F020F81325B5
:10601000061E2DD0029B01240370019B002B04D08F
:10602000001903999847001984B26B461B7A5BB23A
:10603000002B0FDA1021380002F01CFB1925002874
:1060400013D130003219E1B202F066FC051E0CD10A
:106050000C34A4B2042304AA380005A99380069640
:10606000948101F0AFFD051E02D0300005F094FBD5
:10607000280009B0F0BDC0463464FF1F70B50500AC
:106080000C0000280CD00020814209D010222000F2
:10609000044905F029FB01202B7823736B78637387
:1060A00070BDC04604BA0011F0B506000D0017001F
:1060B0001C0085B002291BD00020102907D1022B1B
:1060C00007D0102B03D115E00020102C08D005B00C
:1060D000F0BD69463800FFF7D1FF2A0069460BE0A2
:1060E00069463000FFF7CAFF22006946380004E025
:1060F000022BE9D12A003900300005F055FAE6E715
:10610000031CF02800D9F023032008499AB2013A71
:106110000B80D317034006499B189B100B80D30FAD
:1061200004499B185B100B807047C046AC42FF1FB0
:10613000AA42FF1FA842FF1F034B1B888B4202D3BA
:10614000024B4000C1527047AC42FF1F3464FF1F36
:10615000014B4000185A70473464FF1F1722014B4F
:106160001A8070473464FF1F70B505000E2005F0DB
:1061700083F9041E13D0D0230370002306228370FA
:1061800007494570033005F0AFFA064B2100DA8A63
:1061900062811B7E2373044B187805F04DF870BDA7
:1061A0005064FF1F4064FF1FFC42FF1F262803D8D6
:1061B000024B4000C05A70470148FCE7AE42FF1F47
:1061C000FFFF000070B506000C00094D1C220021E5
:1061D000280005F039FA074B1E70074B1C7005F0BC
:1061E0009BFA0123002801D0002312202B7070BDE0
:1061F0004064FF1FFC42FF1F6164FF1F70B5050074
:106200000D4C0800E260A16010220021656005F0DD
:10621000BBF9012803D11021A06802F058FD10221B
:106220000021280005F0B0F9012803D11021606891
:1062300002F04DFD70BDC0464064FF1F70B5041EE6
:1062400005D1002903D006220D4805F04DFA0D4B6B
:106250001D78012D11D1002C05D102221A7005F0F4
:106260007BFA280070BD00221A70074B1B78FF2BA9
:10627000F7D02000FFF778FFF3E70025F1E7C046ED
:106280005064FF1F4064FF1FFC42FF1F030010B556
:10629000002801D1002010BD00780B4A002803D14E
:1062A0005988D1821B7913761378022BF2D10023FF
:1062B000984200D103331370044B1B78FF2B01D09D
:1062C000FFF752FF0120E6E74064FF1FFC42FF1F7B
:1062D000002911D000280CD04B79012803D140228D
:1062E0005242134303E03F221340032802D001200F
:1062F0004B7170474022F4E70800FAE770B5094D8A
:106300000100287800280BD0074C0622200005F059
:10631000EBF921002878FFF7DBFF200005F064F897
:1063200070BDC0466064FF1F3A64FF1F00290AD099
:10633000012808D13F224B799343C02B03D0403B27
:106340005A425341981C704770B5174D06002B7880
:10635000FF2B15D00A2005F08FF8041E10D0D02393
:106360000370C83B8370114B11491B784670C37092
:106370000622043005F0B8F92100287804F05CFF0B
:106380000C4B1B78012B0DD10B4B1B68002B03D042
:106390009B68002B00D09847084B04211878084AC6
:1063A00005F052F870BDC046FC42FF1F6064FF1F3D
:1063B0003A64FF1F5C64FF1F8864FF1F8C64FF1F2B
:1063C00060EA0000014B98687047C0464064FF1FB8
:1063D000014BDB68186870474064FF1F074B10B51E
:1063E000DA68136801331360054B1878FF2803D06F
:1063F0008021C90105F030F810BDC0464064FF1F80
:10640000FC42FF1FF7B50E0002F0C8F8051E1CD0B5
:106410000E4B06621F78002F00D10778AB79102051
:10642000019305F029F8041E0FD0D0230380C73B49
:106430008370019BE91DC3700622043005F054F9F6
:1064400021003800E66004F0F7FEF7BDFA42FF1FB6
:10645000014B18787047C0466064FF1F054B002849
:1064600005D1054B1A78054B002A00D1014B1800C5
:106470007047C0465064FF1F6064FF1F3A64FF1FEF
:10648000014B58687047C0464064FF1F024B1868B4
:10649000431E9841C0B270476464FF1F421E030050
:1064A0000120152A03D9FF3B5A425341D8B2704705
:1064B000F0B51C0000230E0085B0039002920B7013
:1064C000029A934201D3002019E0E55C5A1CD2B233
:1064D000002DF8D0029851198142F4DC0233DFB26A
:1064E000A35C18000193FFF7D9FF002807D0013DF6
:1064F000019A0399EBB233708A4202D1E01905B0D8
:10650000F0BDDB19DBB2DBE710B50C0002F09EF842
:1065100003001220002B03D02100588804F034FF20
:1065200010BD000070B50E4D84006359002B15D0CE
:10653000186A002801D005F017F92B59586A00286D
:1065400001D005F011F92B59986A002801D005F007
:106550000BF9285905F008F900232B5170BDC046EE
:106560007064FF1F1C4B70B504000E0015009942AB
:106570000AD11A4B1B68002B01D1122070BD1B6879
:10658000002BFAD09847F9E7154B994215D1134BD8
:106590001B68002B0AD01B68002B07D098470028E7
:1065A00004D1104B1C70104B1D70E7E72900200030
:1065B000FFF7AAFF0028E1D1F3E7080001F0EEFFA2
:1065C0000028DAD003780320A342D7D12900300075
:1065D00004F0DAFED2E7C046FEFF00006C64FF1F45
:1065E000FFFF00006964FF1F6864FF1FF7B5040028
:1065F000808801F0D3FF0025A84203D00578A08849
:1066000002F008F81C4E3378002B1FD0AB421DD18E
:106610001A4B28001978FFF777FF002818D00023BD
:106620003370A3790820A778A688019304F024FF8B
:10663000011E0DD0D0230370CA3B8370019B4770AD
:1066400086808371280004F0F7FD01E0002DE8D179
:10665000A0880B4B8200D358002B01D0FFF762FFBC
:106660001721A088FFF768FDA08801F027FDA0880A
:1066700001F0FEFDF7BDC0466964FF1F6864FF1F9F
:106680007064FF1FF0B587B01D000CAB1B880700BE
:1066900001930DAB1B88142002930EAB1B881600D0
:1066A00003930FAB1B880091049310AB1B880593D9
:1066B00004F0E2FE041E1AD0D0230370CB3B4770D7
:1066C0008370C670062229000430002D11D005F019
:1066D0000BF8019B21006381029B0098A381039B1F
:1066E000E381049B2382059BA37404F0A5FD07B0FE
:1066F000F0BD04F0A9FFECE7F7B5009308AB1B88E9
:1067000007000C200D001600019304F0B5FE041ED6
:1067100013D0280001F042FF00280FD00078D023CA
:106720002370C93BA370009B21002381019B6770EC
:10673000A580E680638104F07FFDF7BD014B1878EA
:10674000EDE7C046FC42FF1F13B5040064890389CE
:10675000C2888188C0780094FFF7CEFF13BD000087
:1067600010B5044C2068002803D004F0FDFF00237E
:10677000236010BD7464FF1FA122F0B581889200D0
:106780004A43384B384F1B6804009B189D229200E7
:106790009B18827989B01A603B68002B5FD01D7806
:1067A000324B1B68002B04D05B68002B01D000200B
:1067B0009847260008363100E079FFF7B7FD237DC2
:1067C000E0710200E0780493638A29000393238A2E
:1067D0000293E3890193A38800933300FFF752FFEC
:1067E000E378002B0BD1E289A379A188029201966C
:1067F000E27928000092012201F0DAFEE0703B68A5
:10680000002B20D0FFF7ACFF194D287800281AD0B4
:10681000184B1978FFF778FE002814D02B78E6780B
:1068200008200793A78804F027FE011E09D0D02373
:106830000370CA3B4670837087808671079804F0A6
:10684000FBFC00232B701721A088FFF775FCA088A4
:1068500001F034FCA08801F00BFD09B0F0BD064B3F
:106860009DE7C0463409FF1F7464FF1F8864FF1F43
:106870006964FF1F6864FF1FFC42FF1FF8B5070033
:1068800008000E0001F08AFE041E18D02620FFF733
:106890008DFC051E00D12578062004F0EDFD041EB8
:1068A0000DD00021062204F0CFFED0232370C23B7E
:1068B00021006770A370A680E8B204F0BDFCF8BDAB
:1068C000F0B585B001930AAB1B78070002930BABC0
:1068D0001B7808000D000092039301F05FFE061E76
:1068E00022D0102004F0C8FD041E1DD0102200216B
:1068F00004F0AAFE2620FFF759FC002800D13078CA
:10690000D0232370C13BA370009B21002372019B05
:1069100067706372029BA580A372039BC0B2E3728F
:106920000C9BE36004F088FC05B0F0BDF7B50D00EA
:10693000019001F033FE071E20D00E2004F09CFDD4
:10694000041E1BD02620FFF731FC061E00D13E7826
:10695000D0232380C53B0622A370F91DE01C04F060
:10696000C3FE019B2A0063810123DD401A401D40C4
:10697000210022736573F0B204F05EFCF7BD0000E5
:10698000F0B585B0029010000D0017000A9E039329
:1069900001F004FE041E31D0029B002B2ED1039B7C
:1069A00002795B0724D5122313430422002E08D159
:1069B0000B99002905D10C99002902D10D990029C4
:1069C0001AD01A430D9B2271002B00D0C9E0002E73
:1069D00000D1CFE0002D00D0CCE0606A002801D0CB
:1069E00004F0C2FE1C21300004F056FE606205E097
:1069F00002239A430E33D7E793432371654BBA00C2
:106A0000D458002C00D1AAE0002E10D0236A002B0D
:106A100003D11C2004F060FD20625E4BBA00D35805
:106A2000186A002803D01C22310004F05DFE0C9B84
:106A3000002B12D0574CBB001D596B6A002B03D1A1
:106A4000162004F049FD6862BB00E358586A00282C
:106A500003D016220C9904F047FE0D9B002B11D099
:106A60004C4DBC006659B36A002B03D1142004F0CE
:106A700033FDB0622B59986A002803D014220D9977
:106A800004F032FE380001F089FD051E67D0414B4D
:106A9000BA00D358002B62D01A6A3420002A00D1E1
:106AA0001C389A6A002A01D0143080B20B9A002A4E
:106AB00001D01C3080B25B6A002B01D0163080B24E
:106AC00004F0DAFC041E4AD01822002104F0BCFDB8
:106AD0002620FFF76BFB0190002801D12B78019352
:106AE000D0232370029B200063700A23294EA370D9
:106AF000039BBD00A371AB59A780196A1830002908
:106B000005D01C22A06004F0EFFD20003430735942
:106B1000996A002907D0030014221433E06002931D
:106B200004F0E2FD02980B9B002B08D003001C220E
:106B30001C330B992061029304F0D6FD029873591F
:106B4000596A002903D01622606104F0CDFD6B461E
:106B50002100187904F070FB3800FFF7E3FC05B062
:106B6000F0BD10220D9B0D991B69A018236204F043
:106B7000BBFD2CE70B9B002B00D13FE7012D00D084
:106B80003CE7606A002801D004F0EEFD1C210B9860
:106B90002AE7C0467064FF1F10B5044C2068002827
:106BA00003D004F0E1FD0023236010BD6464FF1FE7
:106BB0000B4B07B51A68002A01D100200EBD6946AB
:106BC000531C012012780731FFF772FC0028F4D023
:106BD00002780123100018401A42EED0EEE7C046BA
:106BE0008064FF1FF0B51F4F01203B6887B0002B6A
:106BF00025D09B78059300F0B3FB002821D00A2014
:106C0000FFF7D4FA04000B20FFF7D0FA164B05006B
:106C10001E78731E9E413B68F6B2191DD878FFF7A7
:106C200057FB3B682900DA7A043303929A7901937F
:106C30000292009033002000059A04F085FD07B011
:106C4000F0BDFFF7B5FF002805D00620FFF7AEFA2C
:106C500004000720D8E70820FFF7A8FA040009205D
:106C6000D2E7C0466464FF1F6064FF1F70B50A4E20
:106C7000040033780D00FF2B0DD0042004F0FCFB42
:106C8000011E08D0D0230370CE3B45708370C470C2
:106C9000307804F0D1FA70BD0C43FF1F70B50400CA
:106CA00006200D0004F0E8FB011E0AD0D02303707B
:106CB000CD3B8370054B44701B688580187804F0C9
:106CC000BBFA002C01D0FFF767FF70BD6464FF1FA3
:106CD000F8B5264F06003B680D001124002B05D1A6
:106CE0000522234B1B78134202D112242000F8BD49
:106CF000204A10241268002AF8D01278002AF5D011
:106D0000DB0719D52B789A1E012A1AD80C2004F01B
:106D1000E3FB132438600028E8D000230A224370E4
:106D200029000670023004F0DFFCFFF75BFF041E51
:106D30000AD0FFF731FFD9E700F012FB0028E1D1BC
:106D4000E4E7002BE2D0D0E70B4B1B78032BCDD12F
:106D50001D20FFF72BFA094B18800028C6D0084BDE
:106D600004211878074A04F06FFBBFE76464FF1F33
:106D70006164FF1F8064FF1F6064FF1F5E64FF1F6C
:106D80008C64FF1F60EA0000F7B50193194B1400F3
:106D90001A78052306000F0012201A4221D001297B
:106DA00020D1154B1D68002D1BD002201F2C18D898
:106DB000002C02D0019B002B13D0104B1F221E7001
:106DC0006E1C0021300004F03FFC019922003000CD
:106DD00004F08AFC310020002C70002F06D004F053
:106DE0008BFAFEBD064B12201D68DCE704F07CFB2D
:106DF000F7E7C0466164FF1F8064FF1F0C43FF1F5D
:106E00007C64FF1FF8B50F4E12243368002B17D097
:106E10001B780F3C834213D100250B4F0221387899
:106E200004F0A2FA094B042138781D8004F09CFA82
:106E3000074B28001D8033685C7004F03DFC0400A3
:106E40002000F8BD6464FF1F8C64FF1F7864FF1F7F
:106E50005E64FF1F70B5012823D11B4C2388002BD3
:106E600003D01A4A1578002D07D0194B1B68002B48
:106E700002D01878FFF7C6FF70BD3B2B02D93C3B10
:106E80002380F9E7134E0221307804F06DFAFA22DC
:106E90002388920002215A43307804F09DFB25801C
:106EA000EAE70B4B1B68002BE6D00B4B1B785B070C
:106EB000E2D5084B0221187804F056FA0022024B62
:106EC0001A80FFF769FED7E77864FF1F5C64FF1F35
:106ED0006464FF1F8C64FF1F6164FF1FF8B51E4DC3
:106EE0002868002803D004F03FFC00232B601B4ED1
:106EF0003068002803D004F037FC00233360184FBB
:106F000005243B7818002040234221D0154800F08A
:106F10002BFA3B78234213D0202004F0DDFA2860BE
:106F2000002813D02022002104F08EFB202004F042
:106F3000D3FA041E306005D02022002104F084FB27
:106F4000002004E0286804F00FFC2C601320F8BD3A
:106F500000F00AFAF4E7C0468064FF1F7C64FF1F5C
:106F60006164FF1F0043FF1F10B50A4C23681A1EFF
:106F70000ED0002808D10130587004F09DFB002885
:106F800005D02368002B02D00021FFF787FE0122E5
:106F9000100010BD6464FF1FF7B5274E050033686D
:106FA0000191181E21D05C78244F012C30D1FFF7BD
:106FB000FFFD002825D02000FFF7F8F80400412845
:106FC00014D91F4B022118781E4A04F03DFA1E4BBB
:106FD0003C3C1C80022233685A703B78002B14D151
:106FE00028000199FFF75AFE0120FEBDFA22920007
:106FF0004243002AEED0124B0221187804F0ECFA3A
:10700000E8E7FFF7D3F80200F3E700233B70EBE774
:107010003B78002BE8D1032004F02EFA011E08D0A3
:10702000D0230370CC3B457083703368187804F02C
:1070300003F9FFF7B1FDD7E76464FF1F5C64FF1F2E
:107040008C64FF1F60EA00007864FF1F10B51749C9
:10705000838802008B4220D011D815498B4217D06B
:10706000144900205B1899B2012907D89268117859
:107070005A425341D8B2FFF7F9FD012010BD0E4A24
:1070800000209B1807229BB29A424041C0B2F5E70C
:1070900083681878FFF768FFF0E7836899785A7873
:1070A000090218781143FFF777FFE7E70A2000008D
:1070B00006200000F8DFFFFFAFDFFFFF014B187075
:1070C0007047C0460D43FF1F10B5064C207001F0FD
:1070D00041FA207804F0F8F80521207800F062FDEC
:1070E00010BDC0468C64FF1F0BB273B50D00002BA2
:1070F00000DBC4E0884B187804F086FB041E0ED039
:107100000378912B0FD0A22B00D1A1E0834B1878EC
:10711000FF2852D0210004F08FF800284DD18020A4
:107120000002684076BD43780F2B76D013D8052B2C
:1071300070D00E2BEAD18088794B98422BD8794BAE
:1071400098421BD8784B9842E0D1A3681878591C14
:10715000FFF774F838E03E2BD8D18378032B74D036
:107160006CD8012B6ED0022BD0D1704B1B68002B3A
:1071700023D05B68002B20D098471EE06C4BC018D2
:107180000C28C3D804F098F81DC2C2150BC20B0B13
:107190000B3223C23C00674BC0180728B6D8664B99
:1071A0001B68002B09D01B68002B06D020009847D5
:1071B0000AE0A3681878FFF7C7F8200004F0D4F9B4
:1071C000ADE7A068FFF762F800289FD0F5E7A36855
:1071D0001B78002BF1D0554B1B68002BEDD01B68A2
:1071E000002BEAD0210055489847EDE74F4B1B682C
:1071F000002BE2D01B68002BDFD021005048F3E7C2
:10720000504B1B68002BD8D05B68002BD5D02100D9
:107210004348E9E7FFF7EAF9CFE780884A4B98420D
:1072200003D04A4B984200D070E7464B1B68002BB6
:10723000C3D05B68002BC0D02100D5E7153B012BE4
:10724000BBD963E7FFF798FAB7E7FFF77DFAB4E732
:107250003F4B1B78042B07D100236A46138001792A
:10726000408800F0C5FCA8E7364B1B68002BA4D073
:107270005B68002BA1D00100364898479DE70124A8
:1072800021420AD0294B1B68002B04D05B68002BDD
:1072900001D000209847012043E78B070AD5264BF1
:1072A0001B68002B04D05B68002B01D0200098479E
:1072B000022036E70421280008400D4200D131E7C2
:1072C000254E3388002B21D0013B9BB23380002B0D
:1072D0001AD1FFF7DBF800280AD0204B1C70164BA0
:1072E0001B68002B04D05B68002B01D0200098475E
:1072F000FFF7C6F8694601F001FD6846FEF7FEFF9C
:107300001D20FEF753FF308004200AE7024B187857
:1073100004F02AF8F8E7C0468C64FF1F0D43FF1FF6
:107320000E20000001200000091000008464FF1FEF
:10733000FEDFFFFFAFDFFFFF8864FF1F0C200000B0
:107340000B2000006C64FF1F0D20000013200000C4
:107350006164FF1FFFFF00005E64FF1F5C64FF1F8E
:1073600010B501F09BF910BD014B18607047C04685
:107370008864FF1F0B880020162B01D817230420D8
:10738000014A13807047C0463664FF1F00207047D3
:10739000074A03001188814207D091880020994252
:1073A00002D101308000101870470020FAE7C04673
:1073B0009464FF1FF0B58F7806000D00C5B01E2F36
:1073C00015D1FFF7E5FF051E03D10024200045B0CD
:1073D000F0BD00223B003100C078009200F0B2FB0B
:1073E0000400A81C00F0D2FBFF23EB70EEE7264B55
:1073F000062403931B78FF2BE8D0182FE6D87B08D0
:10740000224A013BDB0002929A589446002ADDD0C2
:10741000029AD3185B68002BD8D00878002802D1D4
:107420004B78012B02D10624122FCFD107AFAB88A6
:10743000697800976446AA68A047041EC6D1AB7855
:10744000029A5B08013BDB00D318390030005B680F
:107450009847041E0BD1AB78042BB6D0039A3100A9
:1074600010782200009700F06DFB0400AEE76A7808
:10747000002AABD1AA7805A93B88087130000A70B0
:107480004B80FEF747FBA0E71043FF1F14BA001123
:107490001D4B37B5050098420BD000290AD1FFF7E4
:1074A00077FF002805D11948FFF772FF002800D0A8
:1074B000058037BD01291AD1FFF76AFF041EF8D0F5
:1074C00001235B420380A378FF2BF2D0FE2B07D071
:1074D0000023E0781422009329001E3300F032FBD1
:1074E000A01C00F053FB01235B426380E1E702290B
:1074F000DFD1013901F0BEF80028DAD12800FFF70A
:1075000047FF041EDFD1D4E7FEFF0000FFFF0000AD
:10751000022210B5074B52421A80074801325A80A6
:107520009A80DA8000F07EFA044801F025F8002005
:1075300010BDC0469464FF1FB57300119174001113
:107540000388F7B50400002B02D102252800FEBDF8
:1075500042680221137825485268FEF7A5FD0028ED
:107560002ED0234F01253A88002AEFD0802321888E
:107570005B0201259B1A9942E8DC0C2003F0ACFF6A
:10758000061E31D03B8822889C46002318000195B6
:1075900061469DB2491989B2AA421BD8002801D080
:1075A00062443A8000233000082208C0210004F021
:1075B0009BF8104A1368002B13D100251660C5E70D
:1075C0006268022113780C485268FEF76DFD0028AE
:1075D000C7D1BAE760681D014019418101330198A4
:1075E000D6E71A001B68E6E71325AFE782BA001159
:1075F0000E43FF1F9064FF1F80BA0011014B1870EB
:107600007047C0461043FF1F14230A0010B51A40EC
:10761000194204D00122102101F048F810BD4B0698
:10762000F9D4012088434000F8E710B514008B0618
:1076300004D50122102101F039F810BD08230A00F9
:107640001A40194202D14BB2002B0FDA102101F07F
:107650002DF8002808D02300F2331B78002BECD043
:10766000F1342378012BE8D10020E6E703208907D5
:10767000FAD4E2E7F0B51F00184B85B01C68019002
:1076800002910392002C27D1200005B0F0BDA5681F
:107690003301ED186B89019A934211D3029A9342F8
:1076A0000ED8002F04D10A9B002B10D12C00EBE741
:1076B0003B002978039A6868FEF7F6FC0028F2D1AF
:1076C0000136B6B2A388B342E1D82468DAE7A368EA
:1076D0000A9A5B891380E9E70026F3E79064FF1FAD
:1076E00037B50C000A8849880123914217D3002A34
:1076F00015D0651D23792A0002210A48FEF7D4FC23
:10770000102300280BD023796188208800242A00C8
:107710000094FFF7AFFF0A23A04200D02300180017
:107720003EBDC04682BA001113B50A0008884988D8
:10773000012388420BD8002809D000241379053290
:107740000094FFF797FF0A23A04200D023001800FF
:1077500016BD13B50A0008884988012388420BD852
:10776000002809D00024137905320094FFF782FF26
:107770000A23A04200D02300180016BDF0B58BB03C
:1077800003904A8808880E000123824255D30028BE
:1077900053D00023012704AC23700022718813000A
:1077A0000092FFF767FF051E3ED02078002835D1F4
:1077B0002B78022B18D167706A8983000130E31897
:1077C00080005A8069680222201803F08DFF237818
:1077D0000133DBB22370042B19D93B0068890130D7
:1077E00080B2002BD9D01FE00223637012235843CC
:1077F0006A89231804305A8069681022201803F01F
:1078000073FF23780133DBB22370002BE5D10C4AE0
:107810006B899B185A425341DBB2DFE76378012B37
:10782000E4D12B78022BC7D022780A23002A04D077
:1078300021000398FEF798F9002318000BB0F0BD63
:107840000100FFFF0F4BF0B504001868002816D0A8
:1078500083685D89A54207D88288AE18B44203DAEE
:1078600012019A18934201D10068EFE71E005F8968
:107870001036A74204D1002900D00D801800F0BDB9
:107880003300EFE79064FF1F70B505000C00088817
:107890000021FFF7D7FF03000120002B04D02200B6
:1078A0002800197AFFF7C1FE70BDF7B50C0000255E
:1078B00001902300EE331B78AB4201D800200AE090
:1078C0006B00E65A00213000E718FFF7BBFF0028E5
:1078D00002D126800130FEBD017A0198FFF794FEA7
:1078E000002802D03B882380F5E70135EDB2E0E7C0
:1078F00010B5040008880021FFF7A4FF0300012051
:10790000002B03D02000197AFFF77EFE10BD000087
:10791000054B1B68002B01D1180004E09A685289BE
:107920008242F6D1988870479064FF1FF0B50E2709
:10793000002687B0039302ABFF183E8005001F4B63
:1079400040891400984207D02B78013000976A686C
:1079500080B2FFF78FFE060002212B7818486A6874
:10796000FEF7A2FB00280FD06C892000FFF7D0FFA4
:10797000002802D0013C0419A4B2039B002B00D0C4
:107980001C80300007B0F0BD02212B780D486A68DA
:10799000FEF78AFB0028E7D102212B780A486A68A3
:1079A000FEF782FB002807D0002EDED03B88A342E2
:1079B000DBD17489013CDFE76C89DEE7FFFF000063
:1079C00082BA001180BA00117EBA001110B50C0005
:1079D000FFF7DEFC03000220002B0AD0002C00D0B1
:1079E00023609B781720FE2B03D00138FF2B00D19A
:1079F000002010BD73B50D0001A904001600FFF7AB
:107A0000E5FF172805D0002E04D129002000FEF73D
:107A100027F976BD01221021200000F047FE002842
:107A2000F3D0F6E7014B18607047C046A064FF1F13
:107A300037B56B469D1D010004000222280003F0AB
:107A40008BFC2B88B02B0ED12379122B09D123006C
:107A5000FA331B78012B06D10121608800F0E0F891
:107A600001E01B2BF8D037BD10B5054B0421187071
:107A700000F098F8FFF74CFDFEF770FB10BDC04614
:107A8000A464FF1F0020F0B50BB20F0087B0834243
:107A900034DA274B187803F0B7FE051E2BD0037895
:107AA000A02B25D103AE3100FEF7E4F8041E0BD164
:107AB000B378DB0724D51F4B06341B68002B03D09B
:107AC0003100688898470400A868002801D003F0B6
:107AD00063FE002C08D1184A039B1340174A9342B7
:107AE00006D0B3781B2B03D00121688800F098F8EA
:107AF000280003F039FD80200002784007B0F0BD77
:107B00000F4B1B68002B10D0310068889847041E6B
:107B1000DAD07378002BD7D1B27801A90A704B80E4
:107B20000C716888FDF7F6FFCEE70624F1E7C04642
:107B3000A464FF1F9C64FF1F00FFFF0000011200F0
:107B4000A064FF1FF7B50190FC200D0017001E0078
:107B500003F092FC04001320002C12D0B02320006C
:107B60002370089BF4226770658026710830002B13
:107B700008D0190003F0B8FD2100019803F05CFB68
:107B80000020FEBD089903F05FFDF5E710B5041E67
:107B900006D00078FD2803D803F04EFEFF232370A3
:107BA00010BD00000A1F93B210B504000220032B81
:107BB00005D882400020024BD1529B189C7010BD0A
:107BC000C464FF1F0B8870B5043B04000D00022045
:107BD000032B0BD80121200000F04CFD03001420E2
:107BE000002B03D02900200000F0DEFB70BD000058
:107BF00007B51300034A00920A00012100F02CFC93
:107C00000EBDC0462D7E001107B5019203220092E1
:107C1000024B0A00122100F049FC0EBDAB7E0011A0
:107C200007B56B4601AA11800449D880087806334D
:107C3000012802D1190003F0B7FB07BDA564FF1F9F
:107C40000C4B10B518700023FF210B4A13801381D1
:107C500093819380094A5380137051729381937278
:107C6000D174D3821375517703F0BEFC00F0FCF998
:107C700010BDC046D464FF1FC464FF1FA664FF1F6D
:107C8000F0B58DB06B46002003910C229B5E8342C1
:107C900000DBB0E05D4B187803F0B6FD051E00D1A7
:107CA000A4E00378902B00D09DE006AF0100468849
:107CB000380000F013FA79680400002900D19CE034
:107CC0003B88052B6ED13B89032B1CD905AC2000CA
:107CD00000F0A2F86288172A61D83989131D9942E9
:107CE00031D17968237804310291D90738D5607889
:107CF00000F08EF9071E06D0002303712378012BB4
:107D000008D0132B23D0A868002800D178E003F016
:107D100043FD75E06288029909A800F0A6F8029078
:107D2000380000F08BF909AA2378387A01920022F2
:107D300031000092029A00F012F9380000F064F964
:107D4000029B002BDFD0300000F080F9DBE70378E6
:107D5000032BD8D16288029909A800F0D6F8DEE793
:107D6000122B13D1029909A800F0B5F8021EEAD12E
:107D700027498B88002BC6D0887909A923780191DF
:107D800061780091310000F0EAF8BCE7002302AA14
:107D900093833000617809AAFFF72AFFB3E71D4BF0
:107DA0000993F6E7042B02D09A1F012AABD8184A90
:107DB000043B9B00995A0029A5D0D2189078310035
:107DC0003A0000F0AEF800289DD13B88042B03D088
:107DD00001213000FFF724FF012C04D1A8680028FE
:107DE00001D003F0D9FC280003F0BEFB8020039BE8
:107DF0000002434018000DB0F0BD012800D182E719
:107E000001213000FFF70CFFEDE7C046D464FF1FEF
:107E1000C464FF1F010017000B7803704B78437098
:107E2000CB788A781B021343438070470A8803008B
:107E300002700A88120A42700A88012A06D14A880A
:107E400082704A88120AC27004207047022082425F
:107E5000FBD14A8804309A704A88120ADA708A88FC
:107E60001A718A88120A5A71EFE710B504000120CE
:107E700082420CD94B780A781B0213432380834239
:107E800006D1CB788A781B0213436380002010BD93
:107E9000022BFBD1CB788A781B02134363804B798A
:107EA0000A791B021343A380F0E70B8803700B8849
:107EB0001B0A43704B8883704B881B0AC3708B88E6
:107EC00003718B881B0A4371CB888371CB881B0A93
:107ED000C3710820704703000120082A14D14A7892
:107EE0000878120202431A80CA7888781202024384
:107EF0005A804A790879120202439A80CA798879AD
:107F0000120202430020DA80704710B504000120FD
:107F1000022A05D100204B780A781B0213432380E4
:107F200010BDF8B5060010200F00150003F0A4FAEC
:107F300004000120002C0ED0A0230C222900238055
:107F40006780201D002D07D003F0CEFB21003000FC
:107F500003F072F90020F8BD03F076FBF6E7F7B501
:107F60001E00009008AB142017001D78019103F04B
:107F700083FA041E12D0A2230370019B4770438032
:107F8000099B057146710C220830002B07D019009F
:107F900003F0AAFB2100009803F04EF9F7BD099900
:107FA00003F052FBF6E737B5041E0FD04388002BD1
:107FB0000CD00025C1881323007A17220195009563
:107FC000FFF7CDFFFF2365806372257037BD00008A
:107FD00010B50C4904004A88002A09D08B89002B6F
:107FE00005D00020CB8A0222834201D010BD01229D
:107FF00013000A20434300204032C854C81842806E
:108000000472F3E7A664FF1F0023438003707047E8
:10801000094B00211A0010B55C88002C06D01C7991
:10802000844203D10A234B43D01810BD01310A33D7
:108030000329F1D10020F8E7A664FF1F10B5040062
:10804000407A03F0F9FBFF23637210BD70470430E0
:1080500010B580B203F0A8FB002803D004214942E8
:1080600003F062F910BD000070B50025104CA06847
:108070002580A581A580A84202D003F08DFBA560D4
:1080800000250C4C0C4B606D1D80230058331D7077
:10809000A84202D003F080FB6565002560680028D7
:1080A00001D003F079FB013508340A2DF6D170BDFB
:1080B0006C65FF1F1065FF1F6065FF1F70B5041E14
:1080C00009D1054D2880A881A880A868002802D081
:1080D00003F062FBAC6070BD6C65FF1FF0B54B88B0
:1080E00085B00193002343600A7905000F00022A3E
:1080F00000D07BE0CA88032A17D98B685E7819788C
:108100003602DC78D8790E4399781B7A24021B0258
:108110000C43034353495BBA0B80331D93421ED17A
:10812000042C04D0631F022B0ED9012015E0019A04
:108130004D4B1201D35A002B06D00198FFF7BEFF1A
:108140004A4A1369013313610421B8682E812C80D7
:10815000494203F0E9F86860002005B0F0BD434DE6
:10816000042C06D0631F022B0FD9EB680133EB60A0
:10817000DBE7019A3C4B1201D35A002B05D0019842
:10818000FFF79CFF2B6901332B61374B30000293C3
:10819000019B029A1B010193002301998C468B528B
:1081A000130063449C8003939E81FFF750FF039B61
:1081B000041E986016D00421B868494203F0B4F850
:1081C000FA880100043A200003F08EFA0199029A1D
:1081D000FB888A5A043B9B18029A8B522B68013306
:1081E0002B60A2E7AB690133AB619EE71E4B0293A4
:1081F000019B1E01029BF35A002B2DD002998C1972
:10820000A068002828D0012A26D1FA889B189BB2A2
:108210007352A189994217D39B1AC018B96803F009
:1082200063FA029BA289F35A934200D07DE70022B1
:108230002B81A3882B80A3686B60029BF2520B4AB0
:1082400053680133536070E7084A936801339360C1
:108250000198FFF733FF68E7044A5369013353611C
:10826000F6E7C046D664FF1F6C65FF1FDC64FF1F86
:1082700070B5051E15D10B4C0B4B188023005833DD
:108280001870606D002802D003F086FA656525003D
:1082900050356068002801D003F07EFA0834AC4203
:1082A000F7D170BD1065FF1F6065FF1FF0B51700A7
:1082B000A12285B0920001934243394B06001B680E
:1082C0000C009B18D933FF331D78FDF741FF0430B4
:1082D000854204DD3000FDF73BFF0430C5B2BD42EE
:1082E00007D33A0000213000019B03F085FA05B066
:1082F000F0BD2900380003F00FF82300C6B2503358
:108300001E700393019B29006365380002F0FCFF97
:10831000CBB20293002B02D0039B01361E700026C5
:108320002300503303931B78B34204D8606D0028B8
:1083300031D10020DBE7029A2800002A04D0013B5B
:108340001000B34200D02800F700E719387003F09E
:108350005BF8786000280ED03A78019903F0C4F9F0
:10836000019A3B780136D3180E4A0193D369F6B2CD
:108370000133D361D4E7039B18706065A74205D130
:10838000084A1320D36A0133D362B0E7606803F070
:1083900003FA0834F2E703F0FFF900236365C8E746
:1083A0003409FF1FDC64FF1FF7B50D00070004212F
:1083B000686802F0B9FF2B89040003702B891B0A3F
:1083C00043702B8883702B881B0AC3702E8902256B
:1083D0000436F6B2F42E15D81B4B9F4214D10C2054
:1083E00003F04AF81135011E0CD0902303708E3B28
:1083F0000371043B4380154B8460C680187802F0FB
:108400001BFF00252800FEBD5C237B43104AD318C8
:108410000093583301931B78002B0FD103003200D7
:1084200038000099FFF742FF019B05001B78002BE5
:10843000E8D13800009903F047F8E3E7054A07253B
:10844000536A01335362DDE7FEFF0000D464FF1F6F
:108450001065FF1FDC64FF1FF0B587B00090172088
:108460000F0016000193FFF7F2FD1325041E19D02B
:108470000C98031E02D00199201D9847030AE3704F
:10848000052302AAA07004309081277000986670BE
:1084900003A993800494FFF787FF051E02D02000F4
:1084A00003F07AF9280007B0F0BD0000F0B587B0FE
:1084B0001F000CAB1B780391059301210DAB060047
:1084C0001C78049200F0D6F81425002821D0200052
:1084D000FFF77EFD0135041E1BD01149059B0A786C
:1084E00003700132D2B2131EC68001D101231A00DB
:1084F0000B7022713000049B03990097FFF7ACFFCB
:10850000051E09D1230021000648074A093303F05C
:10851000B3F8280007B0F0BD002363802370F8E7AC
:10852000D864FF1FA77F001130750000F8B5050063
:108530000E00064C064F2368002B02D031002800A5
:1085400098470434BC42F6D1F8BDC0467C65FF1F95
:108550009065FF1F0123064A5B425380002313717D
:108560005362044A136053609360D3601361704791
:108570009065FF1F7C65FF1F0200002310B50649B0
:108580009C000859002801D1625010BD0133052B11
:10859000F6D11320F9E7C0467C65FF1F034A5388D4
:1085A000181A434258414042104070479065FF1FDF
:1085B000F0B585B002930AAB1F780CAB1B88009016
:1085C00008000E0001920393FFF7E8FF0500112059
:1085D000002D1BD10E48FFF7E1FF04001520002CF1
:1085E00014D006220B99A771E01D03F07DF8019BC2
:1085F00030002371029B29006371009B6680237009
:10860000039B6562E381FFF791FF280005B0F0BD91
:10861000FFFF000010B5FFF7C1FF04000220002C8F
:1086200012D060880121FFF781FF606A002801D025
:1086300003F09AF828220021200003F005F8012316
:1086400000205B426380207110BD000030B5074AF6
:10865000074C5588010013780020A54204D05B1A0E
:1086600059424B415842104030BDC0469065FF1FF3
:10867000FFFF0000084A10B501230C00904208D00B
:10868000FFF78CFF031E04D0037923405A1E934149
:10869000DBB2180010BDC046FEFF0000024B187987
:1086A000431E9841C0B270479065FF1F70B504002B
:1086B0000D001600FFF772FF002804D10D4B9C42FD
:1086C00000D0143070BD416A03790520002907D01D
:1086D00012221A40102A02D10520002EF2D10F20BA
:1086E000DB06EFD5897E0C20A942894149424942E7
:1086F0000840E7E7FEFF0000030010B5002800D1A6
:1087000010BD0348034A41889142F9D09847F7E7E2
:108710009065FF1FFFFF0000002330B5C45CCD5CF7
:108720006C40D4540133102BF8D130BD0F230022FC
:1087300010B5C45C64002243CA54C25CD209013B38
:10874000F7D210BD0200010010B52032103102F046
:1087500003FF10BDF0B58BB00390102005931700F8
:10876000049102F0B9FE0090102002F0B5FE009BCB
:1087700013240190002B05D000280CD1132400985D
:1087800002F0F2FF019B002B02D0180002F0ECFF78
:1087900020000BB0F0BD102002F09EFE060010205D
:1087A00002F09AFE13240500002E00D1AEE000284E
:1087B00019D01022002102F047FF3200290003984F
:1087C00002F0CAFE041E0ED133787F2B51D8300040
:1087D0000099FFF7ABFF009B1B787F2B53D80199C3
:1087E0000098FFF7A3FF300002F0BEFF002D02D07B
:1087F000280002F0B9FF002CC1D1102002F06CFE5D
:108800000600102002F068FE0290002E7CD00028A6
:1088100078D03A000F3223000125121105D00F3312
:108820003B4015B25A4253411BB26A1E1201002B43
:1088300033D0049BD2B298180099029AFFF76CFFCC
:10884000013D10220021300002F0FEFEADB2049F77
:108850002D017D19AF4242D0002C33D0300002F000
:1088600083FF029B002B00D189E7180002F07CFFF8
:1088700085E729003000FFF759FF28002549009AB5
:10888000FFF74AFFA7E729000098FFF74FFF2800EE
:108890002049019AFFF740FFA5E70F210F400499F7
:1088A0008A18D9B28F4208D9D15C06A8195401336D
:1088B000102BF6D1029A0199C0E7791A484241413A
:1088C000C901F2E73900300006AAFFF725FF3200A0
:1088D000039806A902F040FE10370400BAE7002C06
:1088E000BCD13000029906AAFFF716FF320006A994
:1088F000039802F031FE082204003100059802F0CE
:10890000F3FEABE71324A9E71324AAE7002800D05D
:108910006EE733E788BA0011F0B58BB00F00160090
:108920000225009000283FD0002A3DD00B1DDBB26D
:108930001800029302F0D0FD1135041E34D0FDF76B
:1089400047FD05003A000099201D02F0ADFEEBB294
:108950000393E3702B0CDBB22F0A00936370FFB21A
:108960002B0E2370A7700193FDF72CFD1022010040
:1089700006A802F099FE2100029A04AB06A8FFF7B0
:10898000E9FE051E0DD1039B08223370009B04A94C
:10899000B370019B7770F370301D02F085FEFDF718
:1089A0001DFD200002F0E0FE28000BB0F0BDF0B588
:1089B0008FB00D00149E039004920593002A03D1FA
:1089C000022420000FB0F0BD002EF9D00398FFF76D
:1089D000E5FD1424071EF4D07278337812021A438E
:1089E000B3781B041343F27812061A43036A019208
:1089F000934201D30133E3D1002D03D03B7901240D
:108A00009B07DED50822002106A802F01DFE059B6B
:108A100013240433DBB21800029302F05DFD051E3F
:108A2000CFD0059A0499043002F03EFE04223100B2
:108A3000280002F039FE3900102210310AA802F095
:108A400033FE2900029A06AB0AA8FFF783FE041E34
:108A50000FD1082206A908A802F026FE0822311D1F
:108A600008A802F0A1FD012807D101990398FDF79C
:108A7000C9FC280002F078FEA3E70124F9E7000012
:108A800070B51C4C05002368181E10D0002D14D1A1
:108A90001A78002A0CD1981C083202F025FE02F048
:108AA0004BFC0135002808D123681D70012070BDE2
:108AB0000A331800082202F017FE2368002BF5D0B5
:108AC000122002F0D9FC061E0DD0C12321680370CC
:108AD000457002311022023002F006FE2368310098
:108AE000587802F0A9FB206802F03EFE00232360C4
:108AF000DCE7C046B865FF1FF8B504002020FDF78D
:108B000055FB0D4EA700BB590500002B0DD00028CA
:108B10000BD0D878FF2809D108492A000C55F35901
:108B200007480333611802F0A7FDF8BD290002F0E1
:108B300023FE0028F0D1F8E7D465FF1FBC65FF1FB6
:108B4000519D001170B5064D84006359002B05D06E
:108B5000D87802F071FEFF226359DA7070BDC0460A
:108B6000D465FF1F70B506008CB00C001500002105
:108B70003022684602F068FD31001022684602F09B
:108B800093FD1D2021000322684402F08DFD6846FC
:108B9000FFF7D8FD2D21040003222800694402F0CC
:108BA00083FD20000CB070BDF0B50700160097B033
:108BB00001931CAB1D7830221EAB00910AA8002146
:108BC0001C7802F041FD102239000AA802F06CFD69
:108BD0001022002102A802F037FD0722310002A86E
:108BE00002F062FD072202AB9818631E9C410199B6
:108BF00002F05AFD02AB9C732B005A1E934102AA4D
:108C0000D3730021102206A802F01EFD06221D9932
:108C100007A802F049FD1A2002ABC01806221F99CE
:108C200002F042FD102200990EA802F03DFD102234
:108C300002AB0EA908781C78013A6040D2B20870E5
:108C400001330131002AF5D10AA8FFF77BFD10227C
:108C500012A904000EA802F047FD102206AB0EA9CF
:108C600008781D78013A6840D2B2087001330131AA
:108C7000002AF5D10AA8FFF765FD044310222098C9
:108C8000E4B212A902F010FD200017B0F0BD70B5DB
:108C90000E0014008CB00100102268461D0002F086
:108CA00003FD3100082204A802F0FEFC2100082286
:108CB00006A802F0F9FC6846FFF744FD0400102204
:108CC000280008A902F0F0FC20000CB070BDF8B537
:108CD00006000D0000243719AC4200D3F8BD02F0A5
:108CE000A3FA030A3B70631CDBB201379D4203D930
:108CF0000234F054E4B2EEE71C00EDE773B5060071
:108D00000C000225002819D0002917D0032101A842
:108D1000FFF7DDFF6B469A793F231A400133134377
:108D20006A463000937101A92200FFF71BFF051E60
:108D300004D10322E01C01A902F0D6FC280076BD74
:108D400003785807DA08C00FD20080009B07104351
:108D50009B0F1843C0B2704707230B40C908C900D6
:108D60000B4303707047000070B50400FFF7EAFE84
:108D7000134DA4006359002B21D0186A002801D09C
:108D800002F0F2FC2B59986E002801D002F0ECFCA6
:108D90002B59D86E002801D002F0E6FC2B59186F31
:108DA000002801D002F0E0FC2B59586F002801D0B8
:108DB00002F0DAFC285902F0D7FC00232B5170BDD9
:108DC000D465FF1F0E4B8000C35870B50C00002BFC
:108DD0000FD09D68002D0CD02B78201D0B706B7868
:108DE0004B70A97CFFF7B8FF2B7E23726B69E360A1
:108DF00070BD10220021200002F026FCF8E7C046DA
:108E0000D465FF1F014B18607047C046D065FF1F37
:108E1000074A03008000825810B5002A06D0D08887
:108E2000984203D1012901D1FFF79EFF10BDC04632
:108E3000D465FF1FF0B5264E95B087000B93BB5944
:108E40000500099112200A92002B31D0D888FFF733
:108E5000A5FB04001420002C2AD0280010A9FFF73D
:108E6000B1FFBB591E781D6A002E23D00895FDF76F
:108E7000EFFA07000020FDF7F1FA0790A379E61D4D
:108E8000069310AD0CA9089800F0E2FA0EA928008C
:108E900000F0D7FA0B9B0A990493069B099802935A
:108EA000079B0396019300970EAB0CAAFFF77CFE7D
:108EB00015B0F0BDFDF7CCFA06903000FDF7CEFA04
:108EC000E31DA779079310AB06000893DAE7C046C5
:108ED000D465FF1F30B50C4C85002A59030085B0BE
:108EE0000120002A0ED018006946FFF76BFF2B59AE
:108EF0001A78D888054B002A00D1054B6A4607210D
:108F000000F0D9FB05B030BDD465FF1F43940011BC
:108F10005194001130B5094C8500295985B01022B3
:108F20006846253102F0E0FB2A591121044BD08814
:108F30006A4600F0C0FB05B030BDC046D465FF1FD7
:108F4000ED94001130B5094C8500295985B01022E7
:108F50006846353102F0C8FB2A591121044BD088EC
:108F60006A4600F0A8FB05B030BDC046D465FF1FBF
:108F70002B950011F7B54D4F86001020F4590D00C8
:108F800002F0AAFAF3592062186A132200286CD062
:108F9000033A29009C6802F0A7FBF3591A78019262
:108FA000002A58D11E6A227D317B9446514001220D
:108FB000019F114201D167461740217D91433943FA
:108FC0002175377B4F40BC4660460027800701D49F
:108FD0004F081740012102208F40227D82433A43EF
:108FE0002275377B5740BC4660460027400701D4B6
:108FF00097080F400420227DBF0082433A43227528
:10900000627D002794466046727B42400A4201D14D
:1090100067460F400121627D8A433A436275777B40
:109020005740BC4660460027800701D457080F40D0
:109030000220627D7F00824317436775767B0022A2
:109040007E40760701D4BA080A400426617D92006A
:10905000B1430A4362756A78002A08D06278002A10
:1090600005D005220533DA7700221000FEBD042268
:109070002979114205D1A17C114202D10533033A6D
:10908000F1E7019A21782C78002A02D10A00210008
:10909000140018220429E8D8042CE6D805206043DF
:1090A000034A05331218525CDDE7C046D465FF1F42
:1090B00098BA001110B50A001121024B00F0FBFA1A
:1090C00010BDC046879500110B0030B587B001ADCB
:1090D0002B806B4604001100981D082202F004FB4F
:1090E0002A000B212000024B00F0E5FA07B030BD4A
:1090F000AF95001110B50A001121024B00F0DBFA08
:1091000010BDC0460396001113B50B0011006A464E
:1091100013706B4604000622581C02F0E5FA6A46FA
:1091200008212000014B00F0C6FA13BD2396001160
:1091300010B50A001121024B00F0BDFA10BDC04667
:10914000739600117FB505000B4BAA00D458080098
:10915000002C0FD0666F237FE28821780396266F5C
:109160000296E66E0196A46E0094FDF709FC2800B5
:10917000FFF7FAFD7FBDC046D465FF1F10B517216C
:10918000FFF7E0FF10BD000070B50A000D00064BB0
:109190000221040000F08FFA060029782000FFF772
:1091A000D1FF300070BDC0465395001170B586B038
:1091B00000236A461370836804001D78681E0A281D
:1091C00059D801A902F070F9060633373B3F4347EF
:1091D0004B4F5300180000F042F9062312284BD0E1
:1091E00000281BD16088FFF7D9F90823002813D085
:1091F0004279002A47D1264B1A78072312070BD54C
:10920000244B1A680723002A06D01668002E03D0C4
:10921000290001AAB04703006A4613706B461B7809
:109220006088002B2AD1FFF767FC06B070BD1800DC
:1092300000F06CF9D4E7180000F087F9D0E71800C7
:1092400000F093F9CCE7180000F0ADF9C8E718007A
:1092500000F0C3F9C4E7180000F0F6F9C0E7180001
:1092600000F0F6F9BCE7180000F013FAB8E71800B0
:1092700000F013FAB4E707236A4613706946608862
:10928000FFF782FFD1E70523012AC5D1024BB8E7DA
:109290006164FF1FCC65FF1FD065FF1FF8B52C4F21
:1092A0008600F35904000D00002B40D0DA8882427A
:1092B0003DD15A78062A33D11A78002A2ED00120BF
:1092C00099681A6A097D014206D0157B054203D0D0
:1092D00007225A700120F8BD0220014204D0157BFC
:1092E000054201D00922F4E70420014204D0127B98
:1092F000024201D00B22ECE7164B1B68002BE9D091
:109300005B68002BE6D020009847BB5900215B78B2
:10931000122BDFD12000FFF715FFDBE70E4BECE748
:10932000112A04D1002900D032252900F2E7002DAE
:1093300008D12000FFF732F9002803D0102302796A
:109340001343037121002800FDF798FAC2E7C046D5
:10935000D465FF1FCC65FF1FD065FF1F70B50E4E93
:109360008500AB590400002B13D01B78002B11D1C2
:109370000A4B1B68002B04D05B68002B01D0200037
:10938000984773595B78122B03D100212000FFF717
:10939000D9FE70BD024BECE7D465FF1FD065FF1FFF
:1093A000CC65FF1F094B8000C3581020002B0CD048
:1093B0001A6A002A09D09B68002B06D0127A1B7EFD
:1093C000101C9A4200D9181CC0B27047D465FF1F08
:1093D00070B503000D0014000220002A30D00029CF
:1093E0002ED013700B78081D53704B789370FFF7D5
:1093F000A7FCE070012002212B7A23716B7B0340D4
:1094000063716A7B0A401343042263716E7B1640CA
:10941000334363716E7BF608F600334363712B7B35
:109420000340A371287B014000200B43A371297BDB
:109430000A401343A3712A7BD208D2001343A371BD
:1094400070BD10B50A0001000120FFF7C1FF10BD7B
:1094500010B50A0001000220FFF7BAFF10BD70B579
:1094600006000C000220002E30D000292ED0737888
:10947000201D0B70B3784B70F178FFF76DFC012263
:109480003579257271794B100800134093401040D4
:109490000343881010408000C9080343C9000B43F0
:1094A0006373B1794B10080013409340104003439D
:1094B000881002409200C9081343C9000B432120C1
:1094C0002373FCF773FE854201D2122070BD222067
:1094D000257AFCF76BFE8542F7D823781820042BF9
:1094E000F4D86378012BF1D80020EFE7030010B522
:1094F0000220002909D0002B07D00322481C0A7043
:1095000019000D3202F0F0F8002010BD0300022215
:10951000080010B5002B06D0002904D00E32591CCB
:1095200002F0E2F80022100010BD030010B5022086
:10953000002909D0002B07D00422481C0A7019000A
:109540000C3202F0D1F8002010BD10B5FFF7DEFF9D
:1095500010BD03000220002906D0002B04D00522F4
:1095600000200A701B784B70704703000220002B0C
:1095700008D0002906D05B7800200B70013B082B37
:1095800000D918307047030010B50220002909D017
:10959000002B07D00622481C0A7019000A3202F07C
:1095A000A3F8002010BD10B5FFF7B0FF10BD0200FA
:1095B0000B00022010B500290ED0002A0CD0072184
:1095C0001970118859701188090A997011180822A8
:1095D000D81C02F089F8002010BD03000A00022008
:1095E00010B5002B0CD000290AD0997858780902C0
:1095F00001431180901CD91C082202F075F800204C
:1096000010BD030010B50220002909D0002B07D09F
:109610000822481C0A701900921802F065F8002010
:1096200010BD02000B00022010B500290BD0002A4B
:1096300009D009211970117818185970511C062287
:1096400002F052F8002010BD10B5FFF75FFF10BD0B
:1096500002000B00022010B5002A09D0002907D013
:109660005178197011180622581C02F03DF800209C
:1096700010BD030010B50220002909D0002B07D02F
:109680000A22481C0A701900063202F02DF8002048
:1096900010BD10B5FFF73AFF10BD02000B0002200D
:1096A00010B5002A06D0002904D018005178FFF721
:1096B00053FB002010BDF0B585B017001E006A46B0
:1096C00006230500080091819380FEF7C0FC132457
:1096D000011E02900CD03800B047041E05D12800AE
:1096E00001A9FEF76FFA041E02D0029802F054F8A6
:1096F0002800FFF701FA200005B0F0BDF0B5040026
:109700008BB0019115000021102202A801F09CFFEE
:10971000334EA700B85900283CD0C388A34239D1A2
:109720000378002B36D14278062A18D102000100B6
:10973000553235310C3006ABFFF7A9FA002829D194
:109740002000FFF72FFE020006A902A801F0CCFFBF
:10975000200002A901F0A8FD01200BB0F0BD816E30
:10976000002917D00B8A112A28D19D420ED10198C9
:109770001231093A01F018FF012807D1BB59200026
:109780009D6EFFF70FFE29000200DEE73221200068
:10979000FFF7D8FC2000FEF701FF061E1BD0416A30
:1097A000002918D00B8AAB4215D10822019812313A
:1097B00001F0FAFE01280ED1716A0AE09D42E9D15A
:1097C00008220198123101F0EFFE0128E2D1BB59C5
:1097D000996E8A7EB9E7200001F05EFEBCE7C046C4
:1097E000D465FF1FF0B56B4D87007E5985B0337887
:1097F00002900393002B00D087E0B368346A019392
:109800007078062817D101221B7D134202D0217BDC
:10981000114218D10222134202D0217B114251D1B0
:109820000422134203D0237B134200D08BE0019B20
:109830005A7DEB5991E007380428F8D801F034FE3E
:10984000032E42678300B36E002B03D11C2001F06E
:1098500043FEB066EB599C6E002C1CD010220021F8
:10986000200001F0F1FE0298FFF79CFD01002000AE
:10987000FFF72DFA01F0D8FC2082200008211230D9
:10988000FFF725FA0298FFF78DFDA076EB5921002E
:10989000D888FFF70FFC0822EB591CE0B36E002BB1
:1098A00005D01A00198AF0881232FFF70DFC022247
:1098B000019B197DEB5911423DD0207B10423AD0DB
:1098C000073208E0F488FCF7DBFD01002000FFF719
:1098D00011FC0A22EB595A70029B9C002A595378BA
:1098E000073B042B11D8D088FEF758FE00284ED035
:1098F000C3895A08D2182849029B0298CB542B5985
:1099000041180433254801F0B7FE05B0F0BDFCF75F
:109910009FFD03000120834201D100200393EB59F6
:10992000DE88FCF79BFD039902003000FFF7ECFB9B
:10993000019AEB59117D042211420CD0217B114276
:1099400009D00B22C7E7F688FCF73CFD0100300088
:10995000FFF7EEFB6BE7019A527D01210A4204D02A
:10996000607B084201D00C22B5E702210A4204D0F4
:10997000607B084201D00E22ADE704210A4204D0E8
:10998000627B0A4201D01022A5E71222A3E7FA2245
:109990005200B0E7D465FF1FD865FF1F5B9D001123
:1099A00010B5064B1A780423100018401A4200D054
:1099B0000348FFF727FA002010BDC0466164FF1F6F
:1099C0001443FF1F70B50400FFF7D4FA051E43D1FE
:1099D0002000FFF77FFA234EA400A0598268937CF1
:1099E000DB0708D50321036A1B790B40012B02D149
:1099F000017F0B430377431DD97F8B1E022B0DD8AC
:109A0000022900D00121C088FCF790FF04213359BE
:109A10001A7F59700A431A77280070BD01290CD1AA
:109A200002231022437000210C3001F00DFE30594A
:109A300010213530FFF74BF9EEE70529ECD1022371
:109A4000D118437010220C3001F04EFE042332591D
:109A5000117F0B431377EAE708251828DCD1053D71
:109A6000DAE7C046D465FF1FF0B58BB00591438897
:109A70007E4F9E00F45915000493002C15D1012946
:109A800002D000200BB0F0BD101D57781678FFF7FC
:109A900057F9EB68320002932B7A049901930090F6
:109AA0003B002000FCF70CFFEBE7E388049A9342AD
:109AB00001D00820E6E72378012B00D1D4E0059BF4
:109AC000581E092800D9CFE001F0EEFC05CE0A2986
:109AD000CC506C859AB229000498FFF773FFD1E748
:109AE000200029001022453001F0FEFDB9594B78C5
:109AF000042B02D1013B4B70C3E70B000A00253356
:109B000035320C310498FFF795F90498FFF702FA03
:109B10000522431E9841BB59C0005A70B2E720008D
:109B200029001022553001F0DFFD049B4F4C9D00B1
:109B3000295904980A0006AB55320C31FFF77AF91F
:109B400029591022453106A801F02EFD012808D11F
:109B50000498FFF7F7F90590002804D106222B5945
:109B60005A7005988EE708230593FAE763780C2B63
:109B70007AD1E36E002B03D11C2001F0ADFCE0662E
:109B8000BB59D86E00286FD01022290001F0ACFD1F
:109B9000BB590498DC6EFFF705FC0D22A076BB597B
:109BA0005A706EE7E06E00285ED063780D2B5BD1B3
:109BB0002B8808220382A91C123001F095FDBB59A5
:109BC0009A68517D0222114226D0186A407B1042C9
:109BD00022D00C32E4E763780E2B45D1236F002BA3
:109BE00003D1162001F078FC2067BB59186F0028BC
:109BF00003D01022290001F077FD0F22BB59CFE7D7
:109C000063780F2B30D1206F0622691C103001F0D1
:109C10006BFDBB599A68517D0422114203D0196A29
:109C2000497B1142D5D100210498FFF78BFA28E730
:109C3000636F002B0DD0BB59586F0028F3D0102252
:109C4000290001F051FD0122BB5952425B6F1A619C
:109C5000E9E7142001F040FCBB5960675B6F002B03
:109C6000E9D126E72978DFE707200BE7D465FF1F56
:109C700010B5064C207001F0B7FD06212078FDF7E5
:109C800091FF0348FEF778FC10BDC046E765FF1F53
:109C9000118E001100200BB270B50D00834216DA50
:109CA000264B187801F0B0FD041E0DD00378922BDE
:109CB0000ED0A02B37D0224B1878FF283AD02100A5
:109CC00001F0BAFA002835D180200002684070BD4A
:109CD00043780E2B0BD03E2BEDD18378052B12D081
:109CE000082BE8D181798088FFF7D8FA08E0154B76
:109CF00082889A42DFD183681878591CFEF7C0FE2B
:109D0000002817D1D7E7104B1B785B0712D50F4BF4
:109D10001B68002B0ED09B68002B0BD0C289811DC5
:109D200080889847ECE7FFF741FAA068002801D047
:109D300001F032FD200001F017FCC5E7E765FF1FC9
:109D40000D43FF1F182000006164FF1FD065FF1F37
:109D500010B50078FFF712FA10BD10B50078FFF7C4
:109D6000FDFA10BD0C234343084A10B59B185A68EE
:109D7000002A03D0012901D1904710BD9B68002B18
:109D8000FBD00029F9D19847F7E7C0460466FF1FCA
:109D900001238340094A10B5946B1C439463506BB4
:109DA00098435063D46B20009843012901D12000CF
:109DB0001843D063116B0B43136310BD0080004048
:109DC000F0B500240127154B85B0DA6B144E0392D1
:109DD0001A6C0192DA64019BE3403B4217D0039D69
:109DE000E5403D400295E5B202992800FFF7BAFF31
:109DF000316A736A002908D03900002B01D002991A
:109E000079402800FFF7C4FF01E0002BF9D10134AD
:109E10000C36172CDFD105B0F0BDC04600800040E5
:109E2000E865FF1F064B01215A68C2400A4204D070
:109E30001B68C3401800084070471B6DF9E7C04617
:109E4000008000400122064B8240002903D0D968DF
:109E50000A43DA607047D9689143D960FAE7C0468F
:109E60000038004030B5032444430F4BE25C1B191B
:109E70009C785D7801232D1B0135AB40013BA3404D
:109E8000A140DB430C00122807D808499200521861
:109E9000116819402143116030BD054A11680B401B
:109EA00023431360F8E7C046DFBA001108F0004012
:109EB00014F00040C21F70B5D4B20623092C0BD891
:109EC0000125084C9540002908D00021FFF7CAFF62
:109ED00023682B4323600023180070BD2368AB4325
:109EE000F8E7C04600380040214BF0B51B185B78FE
:109EF000022B21D1032444431E4A1F4EA35C121996
:109F00009478012215008540B76B013CE4B23D43D3
:109F1000A240B563194C122815D89B0000290CD11A
:109F200017495B1899680A439A600123205C154A17
:109F3000834011680B431360F0BD11495B189968A9
:109F400091439960F1E70E4B00290DD159690A43FD
:109F50005A61225C1328E8D00123203A93400A4931
:109F6000086803430B60E7E7596991435961F0E7DB
:109F7000E865FF1FDFBA00110080004024BB00111C
:109F800000F00040A0F00040A4F00040F8B500242C
:109F90001B4E1C4D1C4B1B5D012B1FD1194A926996
:109FA000E2401A420BD00122B25693402200143AEA
:109FB000D2B2022A09D815494A6913434B610134C8
:109FC00002360C35172CE5D1F8BD0022B2560F49E8
:109FD0009200521891680B439360F0E7022BEED188
:109FE000E7B23800FFF71EFF01235840C1B2380026
:109FF000FFF77AFF3800FFF715FF6877DFE7C04605
:10A00000B1BA0011E865FF1FE965FF1F00F00040CD
:10A01000012202388240054B002903D059690A43C6
:10A020005A617047596991435961FAE70038004015
:10A03000F8B50E0001210F008740114A0400D368D3
:10A04000FD43BB43D360831E8B4201D8FFF7E0FF83
:10A0500000212000FFF72EFF0A4A0B4B5168012E0A
:10A0600005D139431B1951605E700020F8BD2940AD
:10A07000516002221C1962709A6915409D61F4E7D3
:10A080000038004000800040E865FF1F012210B545
:10A090008240074B002906D019680A431A60012143
:10A0A000FFF7C6FF10BD196891431960F7E7C04676
:10A0B000008000400C2370B5002543430A4A290064
:10A0C0009B181D70094B04001B185D70FFF7B0FF53
:10A0D0000123A340064928000A681A430A6005497B
:10A0E0000A689A430A6070BD0466FF1FE865FF1F97
:10A0F000348000403080004070B504000E00FF281E
:10A1000013D003250540FFF7D5FF084AA3089B009D
:10A110009B183F22ED00AA40AE40196820009143F1
:10A12000314319600121FFF78DFE70BD18380040E2
:10A13000F8B50C244443134B0500E4186368002B66
:10A1400003D1A3681220002B1AD0022201270E4B44
:10A1500000215B195A7028002770FFF769FF6368B8
:10A160001E1E08D0A3683E00002B04D02800FFF775
:10A1700059FE4640F6B228003100FFF709FE0020E4
:10A18000F8BDC0460466FF1FE865FF1FF7B5C42091
:10A19000FF222B4B80001958002491433F3A0A4379
:10A1A0001A508022274F5202274E1A60274B1D5DFE
:10A1B000002D21D0A31E012B03D80121E0B2FFF70F
:10A1C00027FF012D18D11F4B9B69E3402B4213D071
:10A1D000E3B218000193FFF725FE01000198FFF795
:10A1E00055FFE3B2143B022B1DD801217156184ACA
:10A1F0008D405369AB4353613B7F002B0DD0E5B2DB
:10A200002800FFF795FF2800FFF70CFE7B7F010079
:10A21000834202D02800FFF7A5FD01340C37023637
:10A22000172CC3D1F7BD012100237156F3568D4081
:10A23000074A9B009B189A68AA439A60DCE7C046CD
:10A2400000E100E0E865FF1FB1BA0011E965FF1FFA
:10A2500000F0004010B501210400FFF7E9FE0123E2
:10A26000044A002011194B70A34091690B4393617C
:10A2700010BDC046E865FF1F70B50E001500040054
:10A28000FFF718FF0C236343094A20009B189D60C9
:10A290005E60FFF74DFFF021064B074A8900051E5F
:10A2A0005A5002D02000FFF705FF280070BDC046BD
:10A2B0000466FF1F0000FF1FC19D001170B5134D04
:10A2C00007202C78002C1FD1982221005200280052
:10A2D00001F062F90123C420FF222B700C4B800097
:10A2E0001C635C630B4B1C605C600B4B1958914307
:10A2F0003F3A0A431A50802252021A600D20074A40
:10A30000074900F0A9FF200070BDC046E865FF1FA7
:10A3100000800040A0F0004000E100E08DA10011AD
:10A320008D9F0011030010B50620072B09D8054AA0
:10A33000137001F071F9D7210020034B034A890003
:10A340005A5010BD3C43FF1F0000FF1F8D1BFF1F15
:10A3500070B51D0002240C2910D8094ACA40D20742
:10A360000CD5FBF72FFF041E08D1059A049928008D
:10A37000FBF744FFFCF7B2FDFFF712FB200070BDB6
:10A380001210000030B50D7802232C009C431842B7
:10A3900001D02B431C0008252300AB43284201D0E9
:10A3A0002B00234320241D00A543204201D01C4341
:10A3B00025002A230D70184204D011781E3B0B4350
:10A3C000137030BD0028FCD10C2113788B43F7E7C4
:10A3D000F8B51D0006AB1B88140007AA0E000B2061
:10A3E0001778002B27D10A78022A49D14A68507879
:10A3F00011780002244A08438018042840D801F04C
:10A4000053F803121D1B2300F06800F03DFF021CEF
:10A41000C0B2B84200D93A1CD2B22000F1682A80FA
:10A4200001F062F906E00222F3681B882A8023709B
:10A430001B0A63700020F8BD0622EEE701232B8083
:10A44000F3681B782370F5E7F368002B16D0082219
:10A450002A801A8822701A88120A62705A88A2709A
:10A460005A88120AE2709A8822719A88120A6271D6
:10A47000DA88A271DB881B0AE371DBE72B80D9E75E
:10A4800001202B80D7E7C04600D6FFFFF7B51600A6
:10A490000A781D0008AB1F880C000123022A18D17E
:10A4A0004A685078117800022B4A08438018032824
:10A4B0000FD800F0F9FF02254439E06800F0E4FE0F
:10A4C000C0B20723B84204D37B190193152B02DDD8
:10A4D0000D231800FEBDE0682A003100C01901F00C
:10A4E00003F96B4600209B88E268D0541B4B1B6825
:10A4F000834203D01B68834200D098470023E8E7DB
:10A500000B23002FE5D1022DE2D1737832781B02A4
:10A510001343E2681380114B1B68002BEED01B68BD
:10A52000002BEBD00120E8E70B23002FD1D1062D23
:10A53000CED12A003100E06801F0D6F8DEE70B2327
:10A54000002FC6D1012DC3D132787533012AC0D86E
:10A55000E3681A70D2E7C04600D6FFFFF467FF1F1A
:10A5600070B50C001500072837D800F09DFF0414C3
:10A5700036361B36242E182015290BD8184E1622D5
:10A580000021300001F060F822002900300001F0C5
:10A59000ABF8002070BD18200229FBD11288114BA6
:10A5A0001A80F6E718200829F4D10A000E4829007D
:10A5B00000F0D2FEEDE718200129EBD10B4B10780B
:10A5C0000B49DA69FFF7DEFEE3E718200129E1D144
:10A5D000064B10780749DA6BF4E70220DAE7C04649
:10A5E000DC67FF1FBA43FF1FB043FF1F4043FF1F3D
:10A5F0006843FF1F8843FF1F030010B50020DB07DF
:10A6000004D50721024A034800F08CF810BDC0466B
:10A610003CBB00114043FF1F054A0300106800289F
:10A6200003D082889A4201D1806870470068F6E7BB
:10A63000EC69FF1F0A88030008009A4204D08A8848
:10A6400004309A4200D0002070470000F8B5F22292
:10A6500000230D4F0D4E7968050042433370994237
:10A6600000D07B600A4C0021200000F0EDFF0023A9
:10A670001A007C60AB4202D100203370F8BD013378
:10A680002280DBB2F234F5E7E46AFF1FE26AFF1FC3
:10A69000F069FF1F73B56B46019006006846150010
:10A6A0001980FCF74DFF041E11D1002D0FD07689C3
:10A6B000002E11D00C2000F00FFF00280ED0084A09
:10A6C0000460136886808560002B02D11060200032
:10A6D00076BD1A001B68F7E70224F8E71324F6E7B3
:10A6E000EC69FF1F012100220A4B10B549420A4CB8
:10A6F000198099809A719A70084B207001201980F6
:10A700005A60FFF7A3FF2078FCF778FF0448FDF7B5
:10A7100033FF10BDFC67FF1FEC6AFF1FE46AFF1FD9
:10A72000D1A70011022310B5002802D0FFF7B2FF15
:10A730000300180010BD0000030010B50020DB0767
:10A7400004D50421024A0348FFF7A4FF10BDC04608
:10A7500050BB0011C043FF1FF0B50E2687B0039316
:10A760000CAB1F8802ABF6180500080031000292FE
:10A77000FDF768F804000120002C0FD03088FFF7A7
:10A780004BFF03000E20002B08D05E68002E05D082
:10A7900021002800039B029A0097B04707B0F0BD44
:10A7A0000A4B10B5984207D10122002352420A8079
:10A7B0008B708A808B7110BDFFF73CFF0028FAD0A8
:10A7C00001235B42038000238370F4E7FFFF000056
:10A7D000F8B5050001290AD1134E00243388F22769
:10A7E000AB4219D028001149FFF7DAFF06E0022931
:10A7F00004D10139FDF73EFF0028EDD0F8BD3B0044
:10A8000063437268D018D35A002B09D03A00002154
:10A8100000F01AFF0134E4B2054B1B78A342EED8D6
:10A8200001235B423380DDE7E46AFF1FFC67FF1F03
:10A83000E26AFF1F10B5FFF7FDFE03000020834210
:10A8400000D0987810BD0000F0B589B01C000EABA8
:10A8500080CB03901E8810AB1B78049202930B7A76
:10A860000D00DB0616D42B780593022B24D0049818
:10A87000FFF7D2FE002812D003689C46002B0ED0B2
:10A88000029B2200019329003B0064460398009636
:10A89000A04705E00498FFF7BFFE002802D10E2074
:10A8A00009B0F0BD8368002BF9D00A222900039873
:10A8B00098470028D7D0F3E76B6858781A786B4B25
:10A8C000000210439842D2D8043B984210D2684B01
:10A8D000984242D015D8674BC0180128C7D80B2022
:10A8E000002EDDD1EB681A7859683A80200028E004
:10A8F000614BC018032800D979E000F0D5FD846AC7
:10A90000789E5E4B9842B2D10B20002EC8D1012315
:10A910003B80EB6831001B7823706889013080B27E
:10A92000FCF790FF3A88031E0ED0017802328A1895
:10A930003A80428962704289120AA270596802788C
:10A94000E01C00F0D1FE06E004323A80310004221F
:10A95000601C00F079FE0020A2E70B20002E9FD1A2
:10A96000EB6807A91E8804233B80330A3000267059
:10A970006370FCF767FF051E28D004AB9A890E238D
:10A9800004A95B183E49C668FCF7D0FF00280BD12C
:10A990002B783C486A680599FBF786FB002803D1B1
:10A9A000012304AA5B42D3813278022A06D171685E
:10A9B000201D00F099FE3B8802333B800E2304AA41
:10A9C0009B181B88A3701B0AE370C4E704ABDE81ED
:10A9D000F4E70B20002E00D062E7E9680398FFF748
:10A9E00029FF02233B802070000A6070B3E70B2030
:10A9F000002E00D054E70222EB681B883A802370B7
:10AA00001B0A6370A7E7E86800F03EFCC2B20300CF
:10AA10000720B24200D243E70DD00299DBB2711891
:10AA2000994202DB921BD3B20293029BE9681A009F
:10AA30003B8089195AE70023F6E70B20002E00D04F
:10AA40002EE70722EB683A801A7822705A786270F3
:10AA50005A88A2705A88120AE2701A792271DA882A
:10AA60006271DB881B0AA37175E7C04604290000E8
:10AA70000228000000D8FFFFFFD6FFFF03280000D8
:10AA8000FFFF000080BA0011F0B58DB06B460020CA
:10AA9000089120229B5E83423DDAA64B187800F095
:10AAA000B3FE071E32D00378B02B2CD100790238C8
:10AAB00016281FD800F020FD17001E001E001E00E3
:10AAC00031001E0096001E001D011E0052011E00D6
:10AAD00073011E00CD011E0050021E001E001E004C
:10AAE0008E021E00E302944B94491B8878880B80E9
:10AAF000FBF71AF83800FCF79BFF914B1B68002B03
:10AB000001D038009847380000F02EFD8020089BC7
:10AB10000002434018000DB0F0BDEE22002187482E
:10AB200000F092FD0BAA3B7B7989388900923A00AC
:10AB30000D32FCF79FFD0400804B1B78002C3FD1A9
:10AB400046E0804B788805937F4B4100CB5A0BAE93
:10AB5000073BDBB232880293002301937B4B210039
:10AB600006930093059BFFF76FFE744D002810D1EC
:10AB7000069B3A8A1B889A420BD1380005991230FD
:10AB800000F012FD002804D02B7862899B00EB189E
:10AB90005A80162306A81B18328820007989FCF7F2
:10ABA000C5FE2B7804009A00AA1851880029C3D04A
:10ABB0000133DBB22B70002807D006A9C98A918027
:10ABC000634A12889A42BCD802E00121494291802E
:10ABD000002B04D059497888FAF7DAFF8AE73E89D2
:10ABE0000A2479E000253E89574B06937B88069A14
:10ABF0005B009B5A033B9D4202DB002DF0D05BE0E3
:10AC0000162206A812183B7B798900923A00300080
:10AC10000D32FCF72FFD0590002858D04689017AA7
:10AC20007888FCF7F1FC041E44D1464B78880793E2
:10AC3000069B4100C95A454B0439C9B206AAD28ABB
:10AC400006930291019400930599079BFFF7FCFD81
:10AC5000041E2FD1069B39491A88931C002D26D13A
:10AC60004B807988384B4900CB5A5119033B8B42B2
:10AC700020DD059B31485B8941190B71A91C013509
:10AC8000C9B2EDB2059145191B0A2B71059B2D49DF
:10AC90000433181800F028FD2C4B059A1B88D31894
:10ACA000DDB22C4B9E4205D00136B6B29CE74988F6
:10ACB0009942D6D0002D0CD0204C2800618800F09D
:10ACC000CBFD207021007888FAF772FF12E7059C0F
:10ACD000F0E7002C00D183E77B78142B00D109E743
:10ACE00016493B794E800B700C717888FAF712FF89
:10ACF00000E7162406ABE41821003889FCF7A2FD12
:10AD0000011E00D1B7E1788822880F4C45002C5BEA
:10AD10000A4D013CE4B2029400240F4B01940095CB
:10AD2000FFF792FD041E00D014E129007888FAF79D
:10AD30004FFFDFE6EC6AFF1FAC42FF1F0468FF1FF6
:10AD4000F867FF1FF868FF1F3464FF1FE869FF1FE3
:10AD5000AA42FF1FFFFF00000668FF1F162406AB74
:10AD6000E41821003889FCF76DFD011E00D182E155
:10AD700078882288AE4C45002C5BAE4D013CE4B295
:10AD800002947C89AC4B01940095FFF75DFD041E95
:10AD900000D0DFE029007888FAF724FFAAE6002532
:10ADA000A44B1D803B00F6331B78A24A788807929B
:10ADB000AB4208D99E4B12880693069943005B5A12
:10ADC000013B9A4203DB0799FAF716FF92E6162435
:10ADD0006B00FB18059306ABE418059B210018894E
:10ADE000FCF730FD011E03D1059B01241E8973E78A
:10ADF0007888924B2288069C099343001B5B904EF7
:10AE0000013BDBB20293002300960193099BFFF7FD
:10AE10001BFD041E02D0059B1E895DE77B88069AF8
:10AE20005B009B5A079A108832881218934202DC02
:10AE30001B1A013B33807F4C02303288099900197C
:10AE400000F052FC2388328801359B182380EDB234
:10AE5000A8E70BAA3B7B7989388900923A000D322A
:10AE6000FCF708FC00250590059B002B04D10A2463
:10AE7000002D00D16EE060E0059B7888197AFCF720
:10AE8000C3FB0100041E63D1694C6C4B78880694A7
:10AE90000993069B4400E45A694B063CE4B20BAEAE
:10AEA000328807930294019100930599099BFFF75B
:10AEB000CBFC041E4CD1079B5E491B881A1D002D3C
:10AEC00030D14A80059B5B4C5A8963191A716B1CFF
:10AED0009BB2E318120A1A71162306A832881B18AF
:10AEE00079890598FCF722FDFF21AA1C2E1D033548
:10AEF0000B00059092B2B6B2ADB2002803D006ABFB
:10AF0000DB8AD9B21B0AA218651911712B714C4D3D
:10AF1000301D2A884949201800F0E6FB2B88F618D6
:10AF2000B5B2A1E74988914207D17A8806995200C3
:10AF3000525AEB18053A9A42C4DC3E4C280061880C
:10AF400000F0EAF9207021007888FAF75FFED1E579
:10AF5000002DF2D13E89BFE6162606ABF618310069
:10AF60003889FCF76FFC3D000400FA3500282DD02D
:10AF7000037A9B060CD400227B8939897888009259
:10AF80003A000C32FFF7E8FB041E10D03E8915E0B2
:10AF90003088FFF741FB00281AD08368002B17D0B8
:10AFA0002100122278889847041EE4D0EEE72B781F
:10AFB000002B02D17888FAF739FE00262B78002B77
:10AFC00000D097E5002C00D194E585E60124DDE76B
:10AFD0000E24DBE7162506ABED1829003889FCF7AF
:10AFE00031FC041E47D0037A9B0611D4154A7B8896
:10AFF0001188994203D01448814207D11380134B22
:10B00000F2261D780023D9B2A94221D30924A1E751
:10B010002888FFF701FB00282FD08368002B2CD055
:10B020002100122278889847041EDFD092E7C0469C
:10B030003464FF1F0468FF1F0668FF1FF868FF1FC6
:10B04000E869FF1FE46AFF1FFFFF0000E26AFF1FBD
:10B0500031005943546801336018615A0029D2D134
:10B060003C0008342100F22200F03EFB21007888E9
:10B07000FAF7E4FD3EE501246CE70E246AE71D4B78
:10B080001A887B889A4231D07888FAF7E1FD31E559
:10B09000F223059851684343CD18C95A00291FD09F
:10B0A0003B7A012B0BD16C88AB887888AA1D009461
:10B0B000FFF752FB041E02D000233B722E88F222BF
:10B0C0000021280000F0C0FA00232B80059B0133EB
:10B0D000DBB20593084B05991B78064A8B42D7D8FB
:10B0E00001235B421380002CCED0F5E5002634000E
:10B0F0000596EFE7E46AFF1FE26AFF1F70B50400E0
:10B100000E001500FFF796FA031E08D1310005481E
:10B11000FFF790FA03001120002B02D01C800020C2
:10B120009D7070BDFFFF0000F8B50B4F06003B7827
:10B130000D001400FF2B0ED00A2000F09DF9011E17
:10B1400009D0B1230380002346800371C5800481A8
:10B15000387800F071F8F8BD0144FF1FF7B50F0013
:10B1600008A90600088809A90B240988002821D10C
:10B170000234022B1ED1557813782D021D432B006B
:10B180008B4301937334002B14D1FB6830001900FA
:10B190000093FFF74FFB019C85420BD02A00300043
:10B1A0000099FFF7ABFF041E04D12A003000798913
:10B1B000FFF7BAFF2000FEBDF0B50E7885B0039012
:10B1C0000AA805880120022E0DD14C6827786478E2
:10B1D00024023C43054FBC4205D10398DBB20196E3
:10B1E0000095FFF7BBFF05B0F0BDC0460229000087
:10B1F000034B10B51B68002B00D09847FEE7C046F4
:10B20000F06AFF1F07B501A8FFF7F2FF044A0548DF
:10B210000021121A00F0C0F9F8F7ECFAFEE7C04678
:10B22000F46AFF1F0444FF1F01B40248844601BCB6
:10B23000604700BF2951010001B40248844601BCA7
:10B24000604700BF594F010001B40248844601BC69
:10B25000604700BFDD66010001B40248844601BCBE
:10B26000604700BF0D31FF1F01B40248844601BC96
:10B27000604700BF056A000001B40248844601BC73
:10B28000604700BF8530FF1F01B40248844601BCFF
:10B29000604700BFDD52010001B40248844601BC92
:10B2A000604700BFED4A010001B40248844601BC7A
:10B2B000604700BF311B000001B40248844601BC56
:10B2C000604700BF093BFF1F01B40248844601BC30
:10B2D000604700BF5D17000001B40248844601BC0E
:10B2E000604700BF156B010001B40248844601BCF1
:10B2F000604700BFED3AFF1F01B40248844601BC1D
:10B30000604700BF4D1F000001B40248844601BCE5
:10B31000604700BF090E000001B40248844601BC2A
:10B32000604700BF090E000001B40248844601BC1A
:10B33000604700BF5549010001B40248844601BC82
:10B34000604700BFD91B000001B40248844601BC1D
:10B35000604700BF0124000001B40248844601BCDC
:10B36000604700BF810E000001B40248844601BC62
:10B37000604700BFB352010001B40248844601BCDB
:10B38000604700BF3139FF1F01B40248844601BC49
:10B39000604700BF8D12000001B40248844601BC22
:10B3A000604700BFD532FF1F01B40248844601BC8C
:10B3B000604700BFE117000001B40248844601BCA9
:10B3C000604700BF3555000001B40248844601BC07
:10B3D000604700BF6D30FF1F01B40248844601BCC6
:10B3E000604700BF8552010001B40248844601BC99
:10B3F000604700BFC521000001B40248844601BC7B
:10B40000604700BFF938FF1F01B40248844601BC01
:10B41000604700BF017F000001B40248844601BCC0
:10B42000604700BF9DA9000001B40248844601BCEA
:10B43000604700BF6D36FF1F01B40248844601BC5F
:10B44000604700BFB139FF1F01B40248844601BC08
:10B45000604700BF5952010001B40248844601BC54
:10B46000604700BF0D52010001B40248844601BC90
:10B47000604700BF75A9000001B40248844601BCC2
:10B48000604700BF1D4D010001B40248844601BC65
:10B49000604700BF2124000001B40248844601BC7B
:10B4A000604700BF091B000001B40248844601BC8C
:10B4B000604700BF1D3BFF1F01B40248844601BC2A
:10B4C000604700BF4936FF1F01B40248844601BCF3
:10B4D000604700BF3119FF1F01B40248844601BC18
:10B4E000604700BF3D4B010001B40248844601BCE7
:10B4F000604700BF5522000001B40248844601BCE9
:10B50000604700BF313BFF1F01B40248844601BCC5
:10B51000604700BF3D18000001B40248844601BCEA
:10B52000604700BF6571010001B40248844601BC58
:10B53000604700BF456B010001B40248844601BC6E
:10B54000604700BF4550000001B40248844601BC7A
:10B55000604700BF7139FF1F01B40248844601BC37
:10B56000604700BFE548000001B40248844601BCC2
:10B57000604700BF434D010001B40248844601BC4E
:10B58000604700BFC56D010001B40248844601BC9C
:10B59000604700BF1D4B010001B40248844601BC56
:10B5A000604700BFB70E000001B40248844601BCEA
:10B5B000604700BFCD4C010001B40248844601BC85
:10B5C000604700BF2D2EFF1F01B40248844601BC16
:10B5D000604700BF0534FF1F01B40248844601BC28
:10B5E000604700BF8B52010001B40248844601BC91
:10B5F000604700BF7918000001B40248844601BCCE
:10B60000604700BF3D37FF1F01B40248844601BCBC
:10B61000604700BF2526000001B40248844601BCF3
:10B62000604700BF8D1BFF1F01B40248844601BC68
:10B63000604700BF6DBC000001B40248844601BCF5
:10B64000604700BFF30E000001B40248844601BC0D
:10B65000604700BF154D010001B40248844601BC9B
:10B66000604700BFADAE000001B40248844601BC93
:10B67000604700BF055E000001B40248844601BC7B
:10B68000604700BFA946010001B40248844601BCDE
:10B69000604700BFC51D000001B40248844601BCDC
:10B6A000604700BFF94C010001B40248844601BC68
:10B6B000604700BF4551010001B40248844601BC07
:10B6C000604700BF691F000001B40248844601BC06
:10B6D000604700BFC53AFF1F01B40248844601BC61
:10B6E000604700BFB54C010001B40248844601BC6C
:10B6F000604700BFE94C010001B40248844601BC28
:10B70000604700BFA54F010001B40248844601BC58
:10B71000604700BFE538FF1F01B40248844601BC02
:10B72000604700BF5125000001B40248844601BCB7
:10B73000604700BF3D36FF1F01B40248844601BC8C
:10B74000604700BFC9A9000001B40248844601BC9B
:10B75000604700BF851F000001B40248844601BC59
:10B76000604700BF291C000001B40248844601BCA8
:10B77000604700BF014C010001B40248844601BC8F
:10B78000604700BF5147010001B40248844601BC34
:10B79000604700BF2146010001B40248844601BC55
:10B7A000604700BFD949010001B40248844601BC8A
:10B7B000604700BFE928000001B40248844601BC8C
:10B7C000604700BFEDA5000001B40248844601BCFB
:10B7D000604700BFC94A010001B40248844601BC69
:10B7E000604700BFB14E000001B40248844601BC6E
:10B7F000604700BFC926000001B40248844601BC6E
:10B80000604700BF0519FF1F01B40248844601BC10
:10B81000604700BFF54E010001B40248844601BCF8
:10B82000604700BF1D3AFF1F01B40248844601BCB7
:10B83000604700BF993AFF1F01B40248844601BC2B
:10B84000604700BF1147010001B40248844601BCB3
:10B85000604700BFAD32FF1F01B40248844601BCFF
:10B86000604700BF350E000001B40248844601BCA9
:08B87000604700BFF137FF1F24
:10B878000001010302030303040305020602070291
:10B88800080209000A030B030C020D000E030F0344
:10B89800100311031303140315001600B53B001120
:10B8A800E93B00110000000002000000BAB80011D6
:10B8B800192A0F180A000000F1590000FD240000A1
:10B8C80041460100817C0011959C0011E97000112E
:10B8D800857A00119552001189AA0011E94E0011CC
:10B8E800C53D0011F53E00110000000016160000CD
:10B8F8000200000004B90011F4FFF3FFD2FC0000BD
:10B908003540001100000000000000005475796106
:10B918000042312E36003030313400676974687562
:10B92800622E636F6D2F70767678004254483031FE
:10B93800000000000200000050B90011292A282A3E
:10B94800272A262A252A242A0A180000E2040000A9
:10B958007102000078EC000074400000102700001D
:10B9680060F0000006640000204E000000000000A7
:10B97800050000001F501D00023CB4000001140027
:10B98800160000008102000030313233343536377A
:10B998003839414243444546000000009956001199
:10B9A800ED5600110000000002000000BCB90011B3
:10B9B8006F2A6E2A1A18000001A00000000000007B
:10B9C8006410B71DC8206E3BAC30D9269041DC7698
:10B9D800F4516B6B5861B24D3C7105502083B8ED42
:10B9E80044930FF0E8A3D6D68CB361CBB0C2649B66
:10B9F800D4D2D38678E20AA01CF2BDBDFB349B5F8B
:10BA0800800000800010000000000000EB5C0011C6
:10BA1800757300110F5D00117D770011935D0011A2
:10BA280053770011095E0011297700115B5E001140
:10BA3800F1780011C35E0011F1780011F55E001174
:10BA4800AB780011095E0011E1760011815E0011EA
:10BA5800897800110000000000000000675F0011F5
:10BA680089780011C95F00118D730011052A042A15
:10BA7800012A002A02290328012800280118001891
:10BA88000000000000000000000000000000008727
:10BA98000101020102010102010203030401030181
:10BAA800010101010303020103000D000E00100053
:10BAB800110013001401070108010A010B011C0100
:10BAC8001D02040205020702080219021A021C02DA
:10BAD8001D03010302031700020100050400080703
:10BAE800000B0A001716001D1C01020101050401C4
:10BAF8000E0D011110011413011716011A19020273
:10BB080001020B0A020E0D0211100214130217167D
:10BB1800030504030807030B0A030E0D00010203C3
:10BB280007090A0B0E0F101112141718191A1B1FE8
:10BB380020212200D1A300118DA4001100000000D3
:10BB48000200000086BA001100000000B9B100111F
:0CBB5800000000000200000084BA001190
:020000041FFFDC
:10000000000000002D3D0011C0B80011BCB8001167
:100010003461FF1F0000000000000000000000002D
:1000200000000000000000000000000000000000D0
:1000300000000000000000000000000000000000C0
:1000400000000000000000000000000000000000B0
:1000500000000000000000000000000000000000A0
:100060000000000000000000000000000000000090
:100070000000000000000000000000000000000080
:100080000000000000000000000000000000000070
:100090000000000000000000000000000000000060
:1000A0000000000000000000000000000000000050
:1000B0000000000000000000000000000000000040
:1000C0000000000000000000000000000000000030
:1000D0000000000000000000000000000000000020
:1000E0000000000000000000000000000000000010
:1000F0000000000000000000000000000000000000
:1001000000000000000000000000000000000000EF
:1001100000000000000000000000000000000000DF
:1001200000000000000000000000000000000000CF
:1001300000000000000000000000000000000000BF
:1001400000000000000000000000000000000000AF
:10015000000000000000000000000000000000009F
:10016000000000000000000000000000000000008F
:10017000000000000000000000000000000000007F
:10018000000000000000000000000000000000006F
:10019000F932FF1F5931FF1FC16601000000000046
:1001A000000000000000000000000000000000004F
:1001B000000000000000000000000000000000003F
:1001C000000000000000000000000000000000002F
:1001D000000000000000000000000000000000001F
:1001E000000000000000000000000000000000000F
:1001F00000000000000000000000000000000000FF
:1002000000000000000000000000000000000000EE
:1002100000000000000000000000000000000000DE
:1002200000000000000000000000000000000000CE
:1002300000000000000000000000000000000000BE
:1002400000000000000000000000000000000000AE
:10025000000000000000000000000000000000009E
:10026000000000000000000000000000000000008E
:10027000000000000000000000000000000000007E
:10028000000000000000000000000000000000006E
:10029000000000000000000000000000000000005E
:1002A000000000000000000000000000000000004E
:1002B000000000000000000000000000000000003E
:1002C000000000000000000000000000000000002E
:1002D000000000000000000000000000000000001E
:1002E000000000000000000000000000000000000E
:1002F00000000000000000000000000000000000FE
:1003000000000000000000000000000000000000ED
:1003100000000000000000000000000000000000DD
:1003200000000000000000000000000000000000CD
:1003300000000000000000000000000000000000BD
:1003400000000000000000000000000000000000AD
:10035000000000000000000000000000000000009D
:10036000000000000000000000000000000000008D
:1003700005B20011000000000000000000000000B5
:10038000000000000000000000000000000000006D
:10039000000000000000000000000000000000005D
:1003A0000000000000000000000000000D1BFF1F07
:1003B000000000000000000000000000000000003D
:1003C000000000000000000000000000000000002D
:1003D000000000000000000000000000000000001D
:1003E000000000000000000000000000000000000D
:1003F00000000000000000000000000000000000FD
:08183800006FFF1F4118FF1FA4
:10184000024981F3088802F057FB0000006FFF1F78
:1018500070B500241E491F4A1F484C6308CA1B0567
:101860001B0DE4188242F9D11C4B80228B630021AE
:1018700009201B4B920519621A4B1B4DDA671B4B53
:10188000DA688243DA609A68194802409A60112047
:10189000296002F08DF8112002F06AF880226B6C4A
:1018A000112093436B64EE23DB006343114A1B0C4E
:1018B00013840122104B9A7201F004FC0F4B1B7829
:1018C000002B04D10E4B1021187802F095FA70BD50
:1018D000000005408805054000060540FF010000A6
:1018E00000F0004004E100E0003800403CF000401F
:1018F000FFDFFFFF0461FF1FB861FF1FE663FF1FEB
:10190000E461FF1F10B502F017FA072804D012286F
:1019100008D0022808D010BD044A0420136B0133FC
:101920001363F8E70220F6E71420F4E7DC64FF1FF6
:10193000F8B507000C0026002500503630785135E8
:10194000002804D10300287058342370F8BD29788A
:10195000CA00481E8141A3183800A25C5B68C9B266
:10196000FFF7D0FF00280DD12B78DA00A218013341
:1019700050602B703378044A013B3370136A013393
:101980001362D8E70123DFE7DC64FF1F5C234343D6
:10199000074910B5C9180B0058331B78012B05D126
:1019A000FFF7C6FF034A936A0133936210BDC04636
:1019B0001065FF1FDC64FF1F10B502F0D5FA064A60
:1019C0000121130010CB4942D967044B136002F088
:1019D00003F9200010BDC04600E100E01000100037
:1019E00010B5040002F0C0FA024B1C6002F0F4F8DB
:1019F00010BDC04600E100E0431E5A425341A02200
:101A0000F0B5D2015B421340154D164A40019B18B8
:101A10002A18127E8BB00191002A1BD01A000832BE
:101A2000D46F0022E6B206AFE4B294420EDC28186E
:101A3000C369002B08D0019902AA117106AA049269
:101A400002AA167303A898470BB0F0BD1978B954D1
:101A50000132EAE71A7D1A7806AB01261A70E6E72A
:101A60009C67FF1F00400040F0B5254B040040017B
:101A7000C25C85B0002A2BD01A18117E002927D00D
:101A8000917E002924D01179022921D11689D78885
:101A9000D168F51BADB22A1C102D00D9102292B2CC
:101AA000BE4217D11818012303710023C269C380F5
:101AB00003819A4206D068460321037301710293A1
:101AC00001A890470820002C00D0192001F0FAFA54
:101AD00005B0F0BD013C65426C41A0256442ED01BA
:101AE0002C40084D1B186419074D0633013A92B279
:101AF000AA42EDD01888461C1E80085C2070F5E7CD
:101B00009C67FF1F00400040FFFF00000F220E4BAC
:101B100010B59868104002380A280BD801F0FEFF73
:101B20000D0A0B0A0A110A0A0A0A060002210020FD
:101B3000FFF762FF10BD0121F9E70020FFF794FFD6
:101B4000F8E7DB6FF6E7C046004000400F220E4B7F
:101B500010B59868104002380A280BD801F0DEFF53
:101B60000E0A0B0A0A120A0A0A0A060002210120BA
:101B7000FFF742FF10BD01210800F9E70120FFF740
:101B800073FFF7E7DB6FF5E70090004013B5334CC8
:101B90002378072B3DD8324B1A78324B002A39D1A3
:101BA0008022196852020A431A60252001F0C0FE03
:101BB00020232D4A11680B43802113606B460422B9
:101BC000C90508680733104228D080210422C905BE
:101BD000C86810422ED080212020C905CA688243DF
:101BE000CA6014221A701A78002A2FD18021C905E0
:101BF000C86820320243CA6014221A701A78002A78
:101C000028D11A4B1A7D22785A601D221A70593237
:101C1000DA6013BD1A6816490A40C5E7086802432E
:101C20000A6014221A701A78002ACED01A78013A63
:101C3000D2B2F7E7C8680243CA6014221A70197852
:101C40004A1ED2B21A700029F9D1C4E71A78013AB3
:101C5000D2B2C7E71A78013AD2B2CEE73C43FF1FAF
:101C60000444FF1F3CF000403443FF1F00200040AD
:101C7000FFFFFEFF564B70B51B68012B03D1554A81
:101C8000936D0133936502F087F8534B534A186004
:101C9000534B544C1A600123534A1360534A136048
:101CA0002378002B06D006225149524802F0BCF995
:101CB00000232370504A514B10681B78C1B2002B8F
:101CC0000ED14F4CC0B223785BB2002B4FDB237890
:101CD00024785BB264B21B0424021B191B18136026
:101CE0000B1C50294ED95023464A47491078DBB285
:101CF000FF2202284BD10868444C454D267890437A
:101D00002A78964254D9227824782E78023B5D10A6
:101D1000A31B6B435201D31A10335B1118430860A5
:101D200002F012F9031F012B45D83A4B1B78002B08
:101D300006D0394B1B78002B02D0002001F0C4FFE5
:101D4000A122364B92009978354B4A431B689B1869
:101D5000832292009B181B78033B012B03D8AF20F2
:101D6000400002F059F901222E4BDA8270BD23782F
:101D700024785BB264B2FF33FF341B0424021B19C6
:101D80000138ABE7CAB2022AAED20223ACE7086838
:101D9000254C264D267890432A78964208D92278F9
:101DA00024782D78023B5B10641B63435201B2E739
:101DB0002378DBB2B2E70228D5D11D4B1B78013B5B
:101DC000022B03D91B4B1B78022BCCD16C20C8E70C
:101DD0009809FF1FFC0FFF1F2864FF1FFF3F000033
:101DE000141003402C64FF1F0C100340001003402C
:101DF000D50BFF1F7211FF1FB40003408C09FF1F9A
:101E0000680AFF1F490AFF1F94000340460AFF1F8C
:101E1000470AFF1FF908FF1F2209FF1F300DFF1F90
:101E20003409FF1FBC0BFF1F440AFF1F450AFF1F99
:101E30001C09FF1F2309FF1F10B501F0DDFE002262
:101E4000014B1A8010BDC0462464FF1F10B502F07C
:101E5000B3F8A121054A89009478054A61431268C4
:101E6000044B5218528C1A8010BDC046300DFF1F13
:101E70003409FF1F2464FF1F10B50D4B0D4A9978DC
:101E8000A1239B004B431268D218531DD97F0A4BE4
:101E90001B88994209D2441C07D0C82805D0D269B2
:101EA0005B1A5A43054B5343C01802F02DF810BD7E
:101EB000300DFF1F3409FF1F2464FF1F7102000053
:101EC00070B5244D2B68002B28D002F08DF82B68BC
:101ED000D8402B680400002B27D001F0CDFF2B68E1
:101EE000D8401D4B1D4A9978A1239B004B43126893
:101EF000D118D25C91239B00002A20D0CA5801320D
:101F0000CA50174B17491B680868834214D3D23B49
:101F1000181A012A1AD0144B186070BD02F064F828
:101F2000124B196802F038F8D3E701F0A5FF0F4B08
:101F3000196802F031F8D4E70D495B18E8E7CA5098
:101F40000C4B1B68DB68E418201AE4E7F530FF301F
:101F5000E1E7C0461C08FF1F300DFF1F3409FF1FBB
:101F60009C09FF1F2864FF1FA009FF1F1808FF1FFF
:101F70002DFF3F003064FF1F70B504000D002829BD
:101F800016D10300A433C2881B889B1A0B4A9BB24C
:101F900093420DD906006A3605223100653001F002
:101FA000B3FE002804D13100200001F08DFF70BD88
:101FB0002900200001F050FEF9E7C046FE7F000036
:101FC000F8B50500012001F0C7FE134CA36AA26A10
:101FD0009342FBD1114E336001F03EFF10490300E4
:101FE00008601048426894460F4A17680022BC45B2
:101FF00001D24268BA1A0D4802603268AD18A422B4
:10200000E562606A520302436262094A1278002A5A
:1020100001D00F3B0B60F8BD00F00040340AFF1FF9
:10202000E408FF1F28100040180AFF1F1C0AFF1FAA
:102030001C09FF1F70B580241025E405A3682B43FD
:10204000A36001F0E1FFA368AB43A36070BD000093
:10205000F7B5160080221C001023D205019191686B
:1020600005000B43936000225A4BD7301A6001F0F1
:10207000E3FD9D232A002F009B00EB58CA3201216B
:102080000092FC37002B01D00021009A386801F043
:1020900093FD2900009BCB311A784F4BD3351A6042
:1020A0004B780A781B0213438A7812041A43CB78C0
:1020B0001B061343494A1BBA13604B790A791B026A
:1020C00013438A7912041A43CB7931001B06134358
:1020D000434A1BBA13606B782A781B021343AA7811
:1020E00012041A43EB781B0613433E4A1BBA1360D3
:1020F000019A330213433C4A13603C4B22001B1BE2
:102100009C4603293DDCB3089A0013005142B21AE1
:10211000032A46D1354AE018511A827840781204D1
:1021200000020243E05C043302430A600022FF2BFA
:102130004BDDF0222E4B12011A600F222D4B1A603C
:102140002D4A1368002BFCD00023224A2749136034
:10215000091B321D0B191B68043A180A23706070A2
:10216000180C1B0EA070E3700434002AF2DC8022ED
:1021700010213B68D20501333B6093688B43936029
:10218000F7BD6346D578981893782D061B042B432A
:10219000157804392B43557804322D022B43036004
:1021A000AFE7022A0AD1114AE05C511AE2185278CC
:1021B000120202430A6004339BB2B7E7012AB5D189
:1021C0000A4A521AE15C1160F5E7084959180A6099
:1021D0000433ACE7000004403C00044038000440F5
:1021E00034000440300004400C000440000104406E
:1021F000040004401000044014000440F7B515002A
:1022000080221C001023D2050091916807000B4327
:1022100093600023654AD730136001F00DFD9D23C4
:102220003E009B00F9583B00CA363200FC330029BF
:1022300000D07FE0586801F0BFFC390032785C4B79
:10224000CB311A604B780A781B0213438A78AC466C
:1022500012041A43CB78281D1B061343554A1BBA98
:1022600013604B790A791B0213438A7912041A43CB
:10227000CB791B061343504A1BBA13604B7A0A7A78
:102280001B0213438A7A12041A43CB7A21001B06DD
:1022900013434A4A1BBA1360009A2B021343484A5D
:1022A00013602200474B1B1B0093009BCE785B18EA
:1022B00001938B7836061B0433430E78043833437E
:1022C0004E78043136023343019E33600328ECDC40
:1022D0000321A808431C9B002940800003292BD11F
:1022E0003849E5185E18A9786D78E35C09042D0279
:1022F000294319433160030008330021FF2B2DDDF2
:10230000314B324919600F21314B196001232749A4
:102310000B60304B19680029FCD006211B680B406C
:10232000042B20D080220020D20593680A318B43F1
:102330009360FEBD01217DE7022908D121495D1886
:10234000E1184978E35C090219432960D3E70129C0
:10235000D3D11C495918E35C0B60CCE71948181815
:1023600001600433CAE7002310490B606346002B69
:102370000CDC3B00FC335A68102101325A60802289
:10238000D205936801208B439360D2E7009B9B1892
:102390001B68190A13705170190C1B0ED37004239B
:1023A0005B4291709C440432E0E7C0460000044068
:1023B0003C00044038000440340004403000044035
:1023C0000C0004400001044004000440080F000019
:1023D000100004401400044070B5061E19D00222FB
:1023E0005A4B9B799343012B13D1594B1A78FF2AEF
:1023F0000FD15A78FF2A0CD19A78FF2A09D1DA78BE
:10240000FF2A06D11A79FF2A03D15B79FF2B00D16D
:1024100099E0504B0C201A78012A08D000224E4D2A
:102420001A7029780B00093B042B01D8212070BDBC
:102430004B1F012BFAD9454CA37B042B00D982E01A
:10244000A279032A00D97EE09A1ED2B2012A02D8CC
:1024500060881F2877D9002E56D0012E73D1A0880E
:102460000128E3D0002907D1581E032803D801F022
:1024700055FB121715122E702978481E032811D803
:102480000025364B1D602823237501F0BDFCA842B2
:1024900027D0A580CAE702212970EDE70421FBE7D8
:1024A0000321F9E707390129C0D82D490968C96A0C
:1024B0008906BBD52B4908780028B7D1012A01D954
:1024C000002BB3D102230B708021274D26338901C5
:1024D0002878237501F0D0FB80212878890101F04C
:1024E0008BFC0123A380214B1B78002B0AD0FA22FE
:1024F00080211F4B92001B8809025A431A4B1878FF
:1025000001F0DAFC002092E701F02EFD2B78A68086
:10251000073B012B03D917482E7001F02DFB114BFF
:10252000114C1A78002A06D08021002220788901D7
:102530001A7001F0A1FB01F04FFB80212078090205
:1025400001F09AFBDEE7122071E7C046A60BFF1FE1
:102550006B09FF1F1A09FF1F1C09FF1F4809FF1FF6
:102560003064FF1F2309FF1F1B09FF1F2109FF1FE5
:102570002C09FF1F0010004010B5002901D001F008
:10258000FBFB10BDF7B5604B01919978A1239B002F
:102590004B435E4A060014681022E418D6235B0001
:1025A000E0583623FF33E35C00279343222B41D1CD
:1025B000574B0F3A1A600760012501F07DFB019B24
:1025C0001880E8235B00E35C002B01D0B34258DDA8
:1025D0000023504FFB70AD33FF33E3581A68002AD5
:1025E00003D09B88DB439B071DD03823FF33E35C7C
:1025F000002B18D09B235B00E35C002B13D1D1335D
:10260000FF33E35CB3420EDAA4235B00E15AE01827
:10261000090A023101F018FB23000122FE33013EBA
:1026200001351A87FA70E8235B00E35C002B2AD09F
:10263000A8B2FEBD03683D00002BBED081880430E7
:10264000090A023101F000FBD6235B00E3581F604A
:10265000B2E72300B133BA00FF33985801378188BD
:102660000430090A023101F0EFFAE8235B00E35C71
:10267000BB42EEDCE822F61AED1800235200A35408
:10268000A6E70027F1E7200001F08EFB00281FD00D
:10269000002E1DDD7319882647190193B60020000E
:1026A00001F0C2FB5A308000201840680135818853
:1026B0000430090A023101F0C7FA200001F034FCAD
:1026C000A3590133A351BD4202D0019B9D42E6D1E3
:1026D000114BE35C002BABD095239B00E35C002BFC
:1026E000A6D00E4BE15A0029A2D00D4AA35C994214
:1026F00002D90133A3549BE700231A212000A354DD
:1027000001F0C2FA94E7C046300DFF1F3409FF1FE5
:1027100000140340E010FF1F5A0200007202000084
:102720005E0200000D4970B54A6E0D4CD2038B69F4
:10273000D20BA24206D80B4D0224AA4204D901F0C2
:102740007BFB70BD02246442E21815007E24254004
:102750002242F4D0A3432B438B61F0E700F000400A
:102760000A200000FC1C0000F8B51D4B1D4F1A7814
:10277000002A10D1BA7B002A02D101321A7003E07C
:10278000032AFAD0022AF8D001F03EFB00220120F1
:10279000154B1A70F8BD154B154D1C68154B9E78DE
:1027A00001232B702878C0B200F09EFBBB7B002B6E
:1027B0000BD101F0F9FBA1239B007343E4188323A1
:1027C0009B00E41823782B70E4E7032B02D101F07F
:1027D000DBF9F0E70020022BDCD101F0D5FBEAE7C2
:1027E0001C09FF1FA60BFF1F2309FF1F3409FF1F32
:1027F000490AFF1F300DFF1FF0B587B00EAD2F78CF
:102800000FAD2D780593AC46634614000E4D0CAA0F
:1028100012782E7803930D9B009201932200059B62
:10282000029701F001FA2E70012C01D0042C08D17E
:10283000802206498B889343054A1278D2011343BC
:102840008B8007B0F0BDC0461C09FF1F6C11FF1F35
:102850007809FF1F0B001B3B70B504003020E02BF4
:102860000DD81300E025493BFF3B9BB2ED00AB4286
:1028700005D8034B200019825A8201F00DFA70BD71
:102880008410FF1F10B501F087FA054B00205B682C
:10289000052B04D9034A5268D20200D4980810BD0F
:1028A00000100040FCE100E070B501F05DFB0D4B55
:1028B0001B68FC33DC691D6AFFF7E4FF641984427E
:1028C00004D2094B01241B68002B07D004220024EA
:1028D000064B1A70064A93690133936101F07CF943
:1028E000200070BD3064FF1F9809FF1F2309FF1FE0
:1028F000FC0FFF1F70B50C4D2B68FC335C6A01F0B8
:1029000033FBFFF7BFFF2B680025FC339B6AE318FE
:10291000834204D2054B1B68AB4200D1051B01F07A
:102920005BF9280070BDC0463064FF1F9809FF1F87
:10293000D722044B92009B5810B5002B00D098472B
:1029400010BDC0460000FF1F10B501F0CFF8FFF723
:10295000EFFF2749274BCA6D274C1A4084235B00A1
:102960001343CB65254B1B68186A01F0F5F9244B1E
:10297000244A1A60244B254A1A60A022244B520094
:102980001A60244B187801F0D7FA2000224901F090
:1029900043FA0023A3600233A360204B2049236045
:1029A00003232048A36001F037FA10221E4BFF20BA
:1029B0001A60802252031A60802292031A608022D9
:1029C00012041A6001F080F9012001F005FAFA20E2
:1029D000400001F0A1F9582001F01EFB134801F05E
:1029E0000BFB012001F060FA072001F0ADF910BDEA
:1029F00000F0004000FEFEFF141000403064FF1F96
:102A0000000003400180063DBC0003403408000084
:102A1000A40003404A0AFF1F71020000C30900001E
:102A2000FFFF3F002810004000E100E0307500008B
:102A3000674E336888331B6883F3088801F0A4F974
:102A4000644A6549136800200B401360634B644A75
:102A50001B68934200D1A6E001F0EEFA0221614A20
:102A600013688B431360FFF76FFF5F4B5F4C187861
:102A7000C0B201F099F80023A3600233A3605C4B5D
:102A80000120236001F068F90323A36001F024F919
:102A9000040001F081F9050001F01EF9554B1860A2
:102AA00001F042F9544B1968621A531EA14200D238
:102AB00013008022D203934201D39B029B0A326807
:102AC000D16AC90700D471E04C491C0C09689BB25B
:102AD0004C4359432402090A641803264849FC322E
:102AE00093680A6847489B1A474A0768126847492B
:102AF0009B18474A9A1833409208DB190A60036012
:102B0000042B03D9013233400A6003600E68414947
:102B1000A619300001F040FA3F4F3E493B68C31808
:102B20003B603000019301F04FF83C4E30680818CC
:102B300038493060884205D9019B01333B6001F080
:102B400043F8316001F0B0F8354B1B78002B0DD005
:102B500001F022F9334B621B196812188A4232D2F3
:102B60004919091B091A304801F056F92F4E337ADA
:102B7000002B0ED001F010F9621BF168121891427F
:102B800024D94919091B091A294801F045F90023DC
:102B90003372284B83F3088801F036F8002001F0E7
:102BA0004BFA00F0D9FF01F047FA5CE7DC0199002D
:102BB0000234641A5900641A09214B438033CB4014
:102BC000A408E41889E7FA218900CCE71A49DBE771
:102BD0003064FF1F1CF00040FFFFC1FF0C0AFF1F05
:102BE000B641210310000040490AFF1F14100040A5
:102BF000C3090000100AFF1F340AFF1F380AFF1F15
:102C0000200AFF1F280AFF1F1C0AFF1F240AFF1F9C
:102C1000C4090000710200006008FF1F2C0AFF1F9A
:102C20001C09FF1FE408FF1F00100040740BFF1F6A
:102C30003C10004000000020DC050000A022054BF5
:102C400092009B5810B5002B01D0984710BD00F0A2
:102C50007BFFFBE70000FF1FA122054B92009B5862
:102C600010B5002B01D0984710BD00F06DFFFBE7B9
:102C70000000FF1FA222054B92009B5810B5002BAD
:102C800001D0984710BD00F05FFFFBE70000FF1F79
:102C9000A322054B92009B5810B5002B01D09847FA
:102CA00010BD00F051FFFBE70000FF1FA422054B01
:102CB00092009B5810B5002B01D0984710BD00F032
:102CC00043FFFBE70000FF1F70B501F065F84F4BB5
:102CD000186001F079F90400C30702D401F07CF90F
:102CE00070BD00224A4B1A604A4B187801380428FC
:102CF00029D800F013FF0320181C2400200001F045
:102D0000EBF80128ECD0444C2378042B6ED100F072
:102D10002BFF0028E4D001F097F8582001F07CF94F
:102D200002232370DCE7200000F05EFFE9E72000CB
:102D300001F0F2F8E5E7200000F06EFFE1E7200087
:102D400001F0A2F8DDE701F0FFF80500012808D145
:102D5000324B1B78053B012B03D82000FFF76EFF99
:102D6000D1E72D4B1B78022B01D0052B20D1022D52
:102D700028D12B4B9B7BAB431CD12000FFF76CFF72
:102D8000264B18780128BED16405BCD424492522DD
:102D90004B7B034205D1233A13405A425341263319
:102DA0001A000B7D9342AED9322001F01DF8AAE73C
:102DB000022D07D1194B1B78052B11D12000FFF7ED
:102DC00059FFDDE7012D0BD1012B03D12000FFF7C7
:102DD0005FFF98E7062B03D12000FFF767FF92E71C
:102DE000200000F0B1FE022D8DD1C9E7032B04D1E4
:102DF0000C4B987C01F050F872E7072B00D06FE77E
:102E0000094B987B01F0A8F86AE7C0469C09FF1FB0
:102E10009809FF1F9009FF1F2309FF1F1C09FF1FAF
:102E2000A60BFF1FBC0BFF1FD40BFF1FFA210A4B81
:102E30000A4A49001A640A4A5A500A4A04395A503E
:102E4000094A08319A64094A5A50094A5C315A5071
:102E5000084ADA667047C0460000FF1FF927FF1FC7
:102E6000F528FF1FA928FF1FD923FF1F6927FF1F70
:102E7000791EFF1F4D1EFF1FF7B50B0CFF27012208
:102E8000009300233C001E001D009446019089B26F
:102E900062469A401000084018413618B6B2FF2F1B
:102EA00002D1012E00D19FB2009802401A41AD1804
:102EB000ADB2FF2C02D1012D00D19CB20133102BF9
:102EC000E6D10320012E07D1012D04D1019B24015D
:102ED000E4191C700138FEBD102EFCD10238102DF3
:102EE000F9D00230F7E700008023F7B59C46264B67
:102EF000264F01932649274A274D284C284B022864
:102F00001AD1604638600868264E30408026360365
:102F10003043086001990978002909D11660224AD6
:102F20002A60224A2260E02219689143A03A1BE0FD
:102F30008021C9021160F2E766463E600F68194EB3
:102F40003E408027FF023E430E6001990978002928
:102F50000DD1176001280ED1154A2A60154A22604A
:102F6000E02219689143C03A0A431A60F7BD8021F4
:102F700089021160EEE7E0210F4A02432A600F4AFE
:102F800022601A688A43F0E74B0AFF1FE000034003
:102F9000D80003409000034000000340500003406D
:102FA00040000340FFFFE3FF0280063D804508220A
:102FB0000180063D80660822008006988055082220
:102FC000F8B51E4B80261A680020140034403242A7
:102FD00032D11A681A4F32431A6001223B68063018
:102FE00093433B6000F0B8FE0122164D2B681E4350
:102FF0002E603B680A2613433B608027BF00124BBC
:103000001B683B4211D1013EF6B2FF2E09D17E2250
:103010000E4B1C682B68E40B1440934323432B6036
:1030200005E0082000F098FEE9E7002EEFD18022AD
:103030002B68600893432B60F8BDC046C4F0004085
:103040005CF0004018F0004068F0004060F0004084
:1030500010B500F049FE01215820034A00F08CFF12
:10306000FFF7AEFF10BDC046600AFF1F10B5782203
:103070000021034800F0A0FE00F0F6FE002010BD85
:103080002467FF1F70B5040000F06EFF00230C20C2
:103090000B4A010059438D18515C00290DD0A14203
:1030A00008D1012300246B7000F0DEFD00F094FDD8
:1030B000200070BD01330A2BEBD11224F6E7C04685
:1030C0002467FF1F70B5040000F04EFF00231900B5
:1030D0001D000D4A1078002806D0A0420CD1557072
:1030E00001310C320A29F5D1002B0AD100F0BCFEC7
:1030F00000F072FD002070BD5078461EB0411B18D4
:10310000EEE700F0B1FDF3E72467FF1FF7B5040019
:103110000C20002384460E4D019267465F43E85D14
:103120007E19A04212D000280BD10A4B9C46624661
:103130001B7808331370019B70707C557160B3600D
:10314000FEBD01330A2BE8D10320F9E70720F7E79A
:103150002467FF1F2067FF1F8020F8B5484BC0057C
:103160001B68C1248360474BFF251A680123134362
:103170004361454BA4001A68444B40211A60444BFC
:103180001A68444B1A60444B1A59AA431A51C52273
:1031900092009E58AE433143802699509F583F4934
:1031A000F6010F403E439E509E5880273602360A55
:1031B0003043985080201A5900020A4002431A51A5
:1031C00004341A59364E3F04324080263A431A518D
:1031D0001A5936061202120A32431A5108341A5981
:1031E00080260A4002431A51C32292009F58B446D7
:1031F000AF4337439F509F58294E0F4007439F507E
:103200009F58374080263604374380269F509F586A
:1032100036063F023F0A37439F50C0221F59AF4333
:103220003A431A511A591202120A1643C6221E5163
:1032300092009C58AC4365462C439C509C580025FA
:103240000C4020439850C72080001A58154C11405C
:10325000C02212020A431A50134B1B78DB08AB4200
:1032600001DC0020F8BD2378002B06D0A368002BDA
:1032700000D0984701350C34EEE71220F2E7C04643
:103280003843FF1F3443FF1FB0F000401C67FF1F8F
:10329000B4F000401867FF1F00E100E0FF00FFFFEF
:1032A000FFFF00FF2467FF1F2067FF1F030010B50B
:1032B0001F2809D8072200201340072404490A7850
:1032C000A24313430B7010BD00230620F5E7C04650
:1032D0002067FF1F054B06491B780A6805485B07F6
:1032E00002401B0B134300200B6070472067FF1F39
:1032F0001CF00040FFFFC1FF70B50C25FFF7EAFF8F
:103300000A4B1C780A4BE4086543ED18002C01D1E8
:10331000200070BD2B78002B06D06B68002B00D0EE
:103320009847013C0C3DF1E71220F2E72067FF1FB0
:103330001867FF1F1FB5002102220B0001910091A9
:10334000052000F0D9FC02230B490A681A42FCD17F
:1033500020230393039B5A1E0392002BFAD1074AA2
:103360001368002BFCDA0B246C442000012100F0D0
:1033700013FC207804B010BD90C8004000C8004085
:1033800013B504000A4B0193019B002B01D11120BE
:1033900016BDFFF7CFFF23000340044205D00520F0
:1033A00000F0DAFC019B013BEDE71800F0E7C046B6
:1033B000FFFFFF0707B500F0D7FD80220821D205E7
:1033C000936A0191002B01D10739916202210C4AC5
:1033D00011600199481E01900029FAD10331116052
:1033E000053101910199481E01900029FAD111601F
:1033F000002B02D18022D205936200F0EDFB07BDC5
:1034000000C00040F0B52D4C89B02378002B4FD17F
:10341000FEF7D2FA02232A4F03903A681A42FCD1EF
:1034200020230693069B5A1E0692002BFAD1254EA6
:103430003368002BFCDA0120FFF7A2FF011E02D047
:10344000112009B0F0BD030003220190009005ADEA
:103450009F2000F051FC0321280000F09DFB022377
:103460003A681A42FCD120230793079B5A1E079201
:10347000002BFAD13368002BFCDA0120FFF780FF24
:103480000028DDD10398FEF7ABFAAA786B78110417
:103490001B020B4329780B4363601300113B0A495D
:1034A000052B07D801239340A3600B6001232370F1
:1034B0000020C6E780231B03F6E7C0462043FF1F1A
:1034C00090C8004000C800409808FF1F1E4B30B550
:1034D0005A6818781D4B85B0D31859424B410121C9
:1034E0000093002300F040FC194B1A4A02259A630E
:1034F00000221A6510325A658022C4219D65164B40
:103500001648D202DA6789004258154B80241A40C7
:1035100080231B0413434350642341200393E40599
:1035200000F006FA402000F003FA6562039D6B1E6E
:103530000393002DFAD103236362FFF73BFFA562DB
:10354000FFF760FF05B030BD2C43FF1F95FFFEF76E
:1035500000C80040050001FF04E100E000E100E0D8
:10356000FFFF00FFF0B585B00700FEF725FA022344
:1035700005002D4C22681A42FCD120230093009BA9
:103580005A1E0092002BFAD1284E3368002BFCDA29
:103590000120FFF7F5FE002803D01124200005B01C
:1035A000F0BD234B2360022322681A42FCD1202362
:1035B0000193019B5A1E0192002BFAD13368002B14
:1035C000FCDA0120FFF7DCFE0028E6D1194B1F6072
:1035D000022322681A42FCD120230293029B5A1E26
:1035E0000292002BFAD13368002BFCDA0120FFF79E
:1035F000C7FE0028D1D1104B2360022322681A4253
:10360000FCD120230393039B5A1E0392002BFAD173
:103610003368002BFCDA0120FFF7B2FE041EBCD198
:103620002800FEF7DDF9B9E790C8004000C8004067
:1036300001000006A8C800400180000110B500206C
:10364000FFF790FF10BD000010B5064B18705960D1
:10365000FFF73CFF00211320034AFFF757FD00202E
:1036600010BDC0462C43FF1FCD34FF1FF0B5040032
:1036700085B003920291FEF79FF9882263035B0BEA
:1036800052051A438023DB059D6A8023274F009251
:10369000BA68002601901B039A420CD9F823260031
:1036A0001B041E401C4206D08022214B52025E6247
:1036B00019680A431A60002D0BD100F055FC022254
:1036C0001C4B1A608023DB055A62013A9A6200F0B3
:1036D00083FA0023039A934220D1002D0AD100F0EF
:1036E00043FC144B03221D608023DB055A629D625C
:1036F00000F072FA8023BA681B039A4208D9002EA0
:1037000006D000220A4B0C495A621A680A401A6015
:103710000198FEF765F9002005B0F0BD009A029906
:10372000D2181278CA540133D4E7C0462043FF1F91
:1037300000C8004000C00040FFFFFEFFF0B587B0AA
:10374000029103920400FEF737F9019000F00CFC9F
:10375000802302250122234EDB0535605D629A62DB
:1037600000F03AFA204F3B682B42FCD1202304930F
:10377000049B5A1E0492002BFAD11C4D2B68002B7F
:10378000FCDA0120FFF7FCFD002802D0112007B071
:10379000F0BD2000039A029900F016FB02230400FA
:1037A0003A681A42FCD120230593059B5A1E0592C4
:1037B000002BFAD12B68002BFCDA0120FFF7E0FD8B
:1037C000051EE3D100F0D0FB80230322DB0535602A
:1037D0005A629D6200F000FA0198FEF701F9E0B22A
:1037E000D5E7C04600C0004090C8004000C8004077
:1037F000F0B5802489B00600FEF7DEF8E405A36A80
:1038000002250393029000F0AFFB0123304F3D608F
:103810006562A36200F0E0F92E4C23682B42FCD1D4
:1038200020230593059B5A1E0592002BFAD12A4DA1
:103830002B68002BFCDA0120FFF7A2FD002803D043
:103840001124200009B0F0BD244B2360022322681C
:103850001A42FCD120230693069B5A1E0692002B87
:10386000FAD12B68002BFCDA0120FFF789FD021E3C
:10387000E6D11B4B03211E60030001900090202025
:1038800000F03AFA022322681A42FCD1202307935F
:10389000079B5A1E0792002BFAD12B68002BFCDAEB
:1038A0000320FFF76DFD041ECAD100F05DFB8023ED
:1038B0000322DB053C605A629C6200F08DF9039B99
:1038C000002B01D1FFF776FD0298FEF789F8B8E7E3
:1038D00000C0004090C8004000C800400100000641
:1038E00094C8004007B5000201910422000A01A912
:1038F000FFF724FF0EBD000073B5050005240B4A39
:10390000A3005B429B1819686B46DE1D3000FFF771
:10391000B3FA022804D133782B55013CEFD276BD9F
:10392000052CFCD00128FAD10230F8E71409001167
:103930001F2807D8012380228340D20591680B43BA
:10394000936070473F2808D80123802220388340A5
:10395000D20551690B435361F3E75F28F1D8012386
:10396000802240388340D205116A0B431362E8E796
:103970001F2807D8012280218240C9058B68934304
:103980008B6070473F2808D8012280212038824070
:10399000C9054B6993434B61F3E75F28F1D80122D6
:1039A000802140388240C9050B6A93430B62E8E7E7
:1039B0001F2810D880230200DB05153A1968012A58
:1039C00006D820229143196019680A431A6070478B
:1039D00001228240F6E73F2811D880230200DB0550
:1039E000353AD968032A06D810229143D960D9689C
:1039F0000A43DA60EBE7012220388240F5E75F28CE
:103A0000E5D842238022181A413B8340D205516AEF
:103A100099435162516A0B435362D8E710B50400D1
:103A2000012813D1A022184992050B685B015B099C
:103A300013430B60154B164A19681140154A0A4387
:103A40001A60402219680A431A6010BD0028FCD190
:103A500001000A2000F048FA21000B2000F044FA8F
:103A6000C0220A4B920019680A4340211A601A6862
:103A70008A431A60B022044912060B685B015B0995
:103A800013430B60E1E7C04614F000401CF0004017
:103A90007F00FEFF80FD010072B6074A1368013304
:103AA00013600422054B1A600023054A136080222C
:103AB000D2055360FEE7C0467808FF1FC0F0004003
:103AC000C4F0004005490B68002B05D1044A0A6088
:103AD00004490A60044A13607047C046140AFF1F75
:103AE000841E0000380AFF1FC4F000400023034A70
:103AF0001360034A1360034A1360704754F0004098
:103B000040F1004044F1004002B4714649084900C8
:103B1000095649008E4402BC7047C04602B4714643
:103B200049084900095C49008E4402BC7047C04600
:103B300003B47146490840004900095A49008E44BF
:103B400003BC70470000000001B40248844601BC79
:103B5000604700BFE917010001B40248844601BC78
:103B6000604700BF8552010001B40248844601BC91
:103B7000604700BF01D7000001B40248844601BC81
:103B8000604700BFC1A5000001B40248844601BCE3
:103B9000604700BF75F8000001B40248844601BCCC
:103BA000604700BF3D71010001B40248844601BC7A
:103BB000604700BF8914010001B40248844601BC7B
:103BC000604700BF2144000001B40248844601BCA4
:103BD000604700BF090E000001B40248844601BCE2
:103BE000604700BF9DA9000001B40248844601BCA3
:103BF000604700BF0934010001B40248844601BC9B
:103C0000604700BF8D82000001B40248844601BCB9
:103C1000604700BF7997000001B40248844601BCA8
:103C2000604700BFF535010001B40248844601BC7D
:103C3000604700BF9D6A000001B40248844601BC91
:103C4000604700BF8944000001B40248844601BCBB
:103C5000604700BFC115010001B40248844601BCA1
:103C6000604700BF51B8000001B40248844601BC5F
:103C7000604700BF21A9000001B40248844601BC8E
:103C8000604700BFB352010001B40248844601BC42
:103C9000604700BF53B9000001B40248844601BC2C
:103CA000604700BF116E000001B40248844601BCA9
:103CB000604700BFD544010001B40248844601BCFE
:103CC000604700BFCD0C010001B40248844601BC2E
:103CD000604700BFED6B010001B40248844601BC9F
:103CE000604700BF156B010001B40248844601BC67
:103CF000604700BFED68010001B40248844601BC82
:103D0000604700BF496D010001B40248844601BC10
:103D1000604700BFCD4C010001B40248844601BC9D
:103D2000604700BF8512010001B40248844601BC0F
:103D3000604700BFC166010001B40248844601BC6F
:103D4000604700BFE927000001B40248844601BC77
:103D5000604700BFF90D010001B40248844601BC70
:103D6000604700BF0189000001B40248844601BCDD
:103D7000604700BFC56D010001B40248844601BC24
:103D8000604700BFE9D4000001B40248844601BC8A
:103D9000604700BFC9A9000001B40248844601BCC5
:103DA000604700BFC95C010001B40248844601BC01
:103DB000604700BF71B0000001B40248844601BCF6
:103DC000604700BFB70E000001B40248844601BC42
:103DD000604700BF9573010001B40248844601BCEE
:103DE000604700BF6911010001B40248844601BC6C
:103DF000604700BF6137010001B40248844601BC3E
:103E0000604700BF0D52010001B40248844601BC66
:103E1000604700BFA9D8000001B40248844601BC35
:103E2000604700BF2D6C010001B40248844601BC0C
:103E3000604700BFD9B0000001B40248844601BC0D
:103E4000604700BFD1AE000001B40248844601BC07
:103E5000604700BF6DF6000001B40248844601BC13
:103E6000604700BFBD5C010001B40248844601BC4C
:103E7000604700BFADAE000001B40248844601BCFB
:103E8000604700BF6D0B010001B40248844601BCCD
:103E9000604700BFF935010001B40248844601BC07
:103EA000604700BF4DF9000001B40248844601BCE0
:103EB000604700BFE512010001B40248844601BC1E
:103EC000604700BF8B52010001B40248844601BC28
:103ED000604700BF85C1000001B40248844601BCB0
:103EE000604700BF0134010001B40248844601BCB0
:103EF000604700BF659E001101B40248844601BCC2
:103F0000604700BF0DB2001101B40248844601BCF5
:103F1000604700BF8937010001B40248844601BCF4
:103F2000604700BF0534010001B40248844601BC6B
:103F3000604700BF5976010001B40248844601BCC5
:103F4000604700BFEDA5000001B40248844601BCF3
:103F5000604700BFDD0C010001B40248844601BC8B
:103F6000604700BFC1F7000001B40248844601BCAD
:103F7000604700BF75A9000001B40248844601BC37
:103F8000604700BF0167010001B40248844601BCDC
:103F9000604700BF19FA000001B40248844601BC22
:103FA000604700BF090E000001B40248844601BC0E
:103FB000604700BFE9F6000001B40248844601BC36
:103FC000604700BFF9ED000001B40248844601BC1F
:103FD000604700BFBD0B010001B40248844601BC2C
:103FE000604700BFDD0A010001B40248844601BCFD
:103FF000604700BFE90B010001B40248844601BCE0
:10400000604700BF8D11010001B40248844601BC25
:10401000604700BFDD3F000001B40248844601BC98
:10402000604700BF7912010001B40248844601BC18
:10403000604700BFE94C010001B40248844601BC5E
:08404000604700BF016C0100A4
:104048000200000082BA001101000000B0B800119F
:10405800020000007EBA0011010000008840FF1F26
:1040680002000000B8B8001101000000B461FF1F91
:10407800020000007CBA0011030000002861FF1F45
:10408800120000000200000082BA001101000000C6
:10409800F8B80011020000007EBA0011010000000B
:1040A800F5B800110200000002B900110300000079
:1040B8006361FF1F020000007CBA001103000000CA
:1040C8007861FF1F020000007EBA001101000000A5
:1040D800F4B800110200000000B90011030000004C
:1040E8003961FF1F020000007CBA001103000000C4
:1040F8005A61FF1F0200000082BA0011010000008F
:104108003CB90011020000007EBA00110100000055
:10411800D141FF1F020000004EB90011010000004C
:1041280033B90011020000007EBA0011010000003E
:10413800D041FF1F020000004CB90011010000002F
:104148008061FF1F020000007EBA0011010000001C
:10415800CF41FF1F020000004AB900110100000012
:1041680023B90011020000007EBA0011010000000E
:10417800CE41FF1F0200000048B9001101000000F5
:104188001EB90011020000007EBA001101000000F3
:10419800CD41FF1F0200000046B9001101000000D8
:1041A80019B90011020000007EBA001101000000D8
:1041B800CC41FF1F0200000044B9001101000000BB
:1041C80014B90011020202020202000000000000FD
:1041D80016150000094B0011CD4A001190B90011C5
:1041E80090011D0018001800FFFF070102030405D5
:1041F80006020106000000000000000000000000A8
:1042080000000000000000000000000000000000A6
:10421800030000000200000082BA00110100000043
:10422800B0B90011020000007EBA001101000000C0
:104238008C42FF1F02000000BAB900110100000003
:10424800AE61FF1F020000007CBA001103000000ED
:104258001864FF1F020000007EBA00110100000070
:104268008C42FF1F02000000B8B9001101000000D5
:10427800B061FF1F020000007CBA001103000000BB
:104288001064FF1F1200000000010000000001116F
:10429800FFFF0000504859360000000000000000F1
:1042A8000B000500F0000000B400002800280028DA
:1042B8003075A000A000A000A00000080008E001E0
:1042C800F000100010001000100010001000500046
:1042D8005000500010001000D0070000000000003F
:1042E8000F0001000500307507001000010081FF74
:1042F80000000000FF0000004D700011556E001115
:10430800E56B0011FFFF0100FF000000699A001132
:10431800E5970011FD960011000000000000000064
:1043280000000800040000003B0001085902E001F9
:1043380088212800FF0000000200000082BA001156
:104348000100000048BB0011020000007EBA001105
:1043580001000000BD43FF1F020000007ABA0011EF
:1043680001000000DC67FF1F020000007EBA001198
:1043780001000000BC43FF1F0200000078BA0011D2
:1043880001000000BA43FF1F020000007EBA0011BE
:1043980001000000B843FF1F0200000076BA0011B8
:1043A80001000000B043FF1F180018001D00900115
:1043B80002000003020200000200000082BA00119D
:1043C800010000005CBB0011020000007EBA001171
:1043D800010000000044FF1F0200000074BA001131
:1043E8000000000000000000020000007CBA00117C
:0A43F80003000000FC67FF1F20FF18
:040000051FFF184180
:00000001FF
